:100000000C9454070C947A070C947A070C947A0792
:100010000C947A070C947A070C947A070C947A075C
:100020000C947A070C947A070C94CF480C94EA4805
:100030000C947A070C947A070C947A070C947A073C
:100040000C947A070C947A070C947A070C947A072C
:100050000C947A070C947A070C947A070C947A071C
:100060000C947A070C947A070C947A070C947A070C
:100070000C947A070C947A070C947A070C947A07FC
:100080000C947A070C947A070C947A070C947A07EC
:100090000C947A070C947A070C947A070C941F4FEF
:1000A0000C94594F0C94934F0C94CD4F0C947A07A9
:1000B0000C947A070C947A070C947A070C947A07BC
:1000C0000C947A070C947A070C947A070C947A07AC
:1000D0000C947A070C947A070C947A070C947A079C
:1000E0000C947A070C947A070C947A070C947A078C
:1000F0000C947A070C947A070C947A070C947A077C
:100100000C947A070C947A070C947A070C947A076B
:100110000C947A070C947A070C947A070C94374E57
:100120000C94714E0C94AB4E0C94E54E0C947A07E3
:100130000C947A070C947A070C947A070C947A073B
:100140000C947A070C947A070C947A070C947A072B
:100150000C947A070C947A070C947A070C947A071B
:100160000C947A070C947A070C947A070C947A070B
:100170000C947A070C947A070C947A070C947A07FB
:100180000C947A070C947A070C947A070C947A07EB
:100190000C947A070C947A070C947A070C947A07DB
:1001A0000C947A070C947A070C947A070C947A07CB
:1001B0000C947A070C947A070C947A070C947A07BB
:1001C0000C947A070C947A070C947A070C947A07AB
:1001D0000C947A070C947A070C947A070C947A079B
:1001E0000C947A070C947A070C947A070C947A078B
:1001F0000C947A07485454502F312E30203230302E
:10020000204F4B0A5365727665723A20776C705FA7
:1002100068747470640A436F6E74656E742D7479BB
:1002200070653A20696D6167652F6769660A0A0023
:1002300047494638396145017B00A10000FFFFFFB7
:10024000006699000000FFFFFF21FE114372656107
:1002500074656420776974682047494D50002C000C
:1002600000000045017B000002FE848FA9CBED0F4A
:10027000A39CB4DA8BB3DEBCFB0F86E24896E6891A
:10028000A6EACAB6EE0BC7F24CD7F68DE7FACEF760
:10029000FE0F0C0A87C4A2F1884C2A97CCA6F3095A
:1002A0008D4AA7D4AAF58A6505B6DCAEF70B0E8B8E
:1002B000C76471F60C2DABD7EC36190D3FBAE7F4D5
:1002C000FA3B8EFFD9F77C7BFE9FD32738C80668A0
:1002D000384398A81876D8D8B2081919E048792276
:1002E00079A958A92982D929B809DAE139CA176A3E
:1002F0008A419A4A77CA3AA1FAEAD62AEB005BAB5E
:10030000368BAB60BB6B96EB0BC01BECF5EB2B6C31
:10031000BC458C7B6C9C3CBB2CDC2CFB1C1CDD3A58
:10032000CD5BCD7ABD9B7DBA6DDB6DFA5D1B1E3A50
:100330000E5B0E7AFE9ABEB9AEDAAEF99E1A5F393E
:100340004F5A4F793F9AEFB8EFD9AFD1BF4E010F57
:100350000DC454D0D0C14B09012D94D4F0CFC34863
:1003600011F34C845411CF1DFE5D601A8CF158A618
:10037000421B04024A9A14B0E0E4C9942A511E6850
:10038000290366B88D091831B0F980A6AB5B2465E6
:10039000F6F4F9122800A12D8836D3790027C76119
:1003A000123E5EE01954A5829625A70A35BA022BA3
:1003B00031A40694D664DAB4D7539D5413503569EA
:1003C000F6AAD4185A7F7105D6F126D8B0715139E2
:1003D0008DBAF26759BD68F9BA84D1B6D8DDAF5F7E
:1003E0004072913B6969E10C64D59E4DBB7647E054
:1003F0005C6FBD22987B199962CC490FD3128BB7E1
:10040000AF81B355FDFA98AC6C70E6C50B58AFDE02
:10041000CCB96B6CD996F70E255DFA76E4D07F47A0
:10042000FBCCCB127883C9A879E77EF0B847E5BA50
:10043000B05B2726CC7C7517C4D17503C79DDB360E
:100440006FC82B8962EFCDFD7878ED56B10FFFCEE6
:10045000E3ADC8D9CE414BF7DCDEB5EFC8E8E70B1A
:10046000B72FBE2CD0EFF7FEF183F78F5B70FC95B2
:10047000376020AAD9C5DE7BD5D1361D75B1FD66A2
:100480001E8004E6572080018E2760851692365E16
:100490008438A847C182D0B9D7197B245A87964C93
:1004A0002AEEB69D5FDAF1C7228AFFC1789F63C248
:1004B000D9289A0D20EE045F4E21C5D7E3880D762A
:1004C00028A37F32FE57A48B10C6481E8EE21D69FA
:1004D000DA04C5DDB0235DCF41009F8822C2B5A0FC
:1004E0007E6BC1449E914A228995931866D85B9889
:1004F000E7C5E84395110489E0950ACA39A7661D46
:10050000DAA6618BC62179248C51EE59619E63F67F
:10051000F7E1810C0EB91407B36D79629F377A78D1
:10052000E69E0CD0B81F8B94EE46239A1CEAB09C32
:100530007C9921C6239D87DA091B9C1BE658DF8422
:10054000E0A9792AA44E663A289BB016DAA8659DE0
:1005500001F926A2733A385BAA8EE6F8A784935E67
:100560008AAAA5C43EF9FE2BA1C9024B43A7268A3D
:10057000EAA990BC1A2622A4AD0E5BA356AC3A6041
:10058000A6079B22F76D0DCEEAFA2990A46E469D30
:100590008FB69EAA2A9B491AB7A6B2DC1AEB6E0642
:1005A00053BEABA3A15C3E6B188F1BE8FB6BBBCCAF
:1005B000EA29ACA6AB762BA98B146CABAA81B53219
:1005C0002A2A63115BB9E58583C64B61BDCB7AC727
:1005D00024B109EB991CC1E2EABB2E971E984A711F
:1005E000C521DFC927BE50622C28C794B21CAEC7F4
:1005F000B4AE5B32B916E89CAB7AE18E093391F365
:10060000FAD9B0C02BB7FAAAC554920C31CAEDBDC5
:1006100037D68FD8BAFB73B02F83AB74A4460F0CB8
:1006200028D5828EFC70B4A34EBC6F8309960AF065
:10063000D59A0E0D2CC345B38DACD0111C0D73CBC8
:10064000F95E94484671E09D89DE68F09DB7DF67EA
:10065000004E88E08313FE89E158209EB8E25630B0
:10066000DE87E35740AD5E8AE45550BE87E5976369
:100670005E87E65470DEB9E75280BE8AE851903E4C
:1006800087E9A7A33E92EA4FB0DEBAEB4DC05E8881
:10069000ECB3D30E95ED4AE09EBBEE48F02EB5EFDD
:1006A000BF039FB6F040105FBCF16D225FB2F27ADB
:1006B00030BFA5F3CB437FB6F43B505FBDF59C62E2
:1006C000EFB4F6CA714FB6F7D7832F3E11E4976F98
:1006D0003EF6E8A74FFDFAEC23EF7E11CCC72F3F83
:1006E000F1F41B01FCFDC3B3AE7F12A4F77F3BC640
:1006F00001F0730719A0010F88C0042A70810C6CE7
:10070000A0031F08C1084A708214ACA0052F8841BD
:10071000CD1500003B485454502F312E302034303A
:10072000342046696C65206E6F7420666F756E6448
:100730000A5365727665723A20776C705F687474DC
:1007400070640A436F6E74656E742D747970653AC7
:1007500020746578742F68746D6C0A0A3C68746D37
:100760006C3E3C686561643E3C7469746C653E6FC8
:10077000574C207069636F2048545450205765626D
:10078000207365727665723C2F7469746C653E3CAB
:100790002F686561643E3C626F64793E3C68323E1E
:1007A000343034202D2050616765206E6F742066D0
:1007B0006F756E643C2F68323E3C703E536F7272B0
:1007C000792C20746865207061676520796F7520C9
:1007D0006172652072657175657374696E672077E3
:1007E0006173206E6F7420666F756E64206F6E206B
:1007F00074686973207365727665722E3C2F703E43
:100800003C2F626F64793E3C2F68746D6C3E0048EB
:100810005454502F312E3020323030204F4B0A5359
:1008200065727665723A20776C705F687474706474
:100830000A436F6E74656E742D747970653A207416
:100840006578742F68746D6C0A0A3C21444F4354D8
:100850005950452048544D4C205055424C49432056
:10086000222D2F2F5733432F2F4454442048544DCB
:100870004C20342E3031205472616E736974696F6C
:100880006E616C2F2F454E222022687474703A2FAF
:100890002F7777772E77332E6F72672F54522F680A
:1008A000746D6C342F6C6F6F73652E647464223EAC
:1008B0003C68746D6C3E3C686561643E3C74697470
:1008C0006C653E6F574C207069636F2048545450DC
:1008D00020576562207365727665723C2F74697467
:1008E0006C653E3C2F686561643E3C626F647920B4
:1008F0007374796C653D666F6E742D66616D696C9D
:10090000793A617269616C3E3C7461626C653E3C2F
:1009100074723E3C74642077696474683D2231309F
:1009200030223E3C2F74643E3C74643E3C746162F1
:100930006C653E3C74722076616C69676E3D227412
:100940006F70223E3C74643E3C696D672073726335
:100950003D226C6F676F2E6769662220616C743D63
:10096000226C6F676F22207469746C653D226C6F16
:10097000676F223E3C2F74643E3C2F74723E3C7481
:10098000723E3C74642077696474683D223530306F
:10099000223E3C68323E576562205365727665722E
:1009A0002072756E6E696E67206F6E206F574C20D7
:1009B0007069636F3C2F68323E3C703E546865201E
:1009C0007765622070616765206973207365727650
:1009D000656420627920776C705F6874747064203D
:1009E0007573696E672074686520482644205769CE
:1009F00072656C65737320574C414E206D6F647542
:100A00006C6520616E6420746865206F574C2D7092
:100A100069636F26636F70793B20536F66747761EB
:100A20007265204150493B206120756E6971756582
:100A30002057692D466920736F6C7574696F6E203D
:100A400066726F6D203C623E4826616D703B4420AB
:100A5000576972656C6573732041423C2F623E2E6C
:100A60003C2F703E3C68723E3C7461626C653E0097
:100A70003C74723E3C74643E49502041646472652B
:100A800073733A20003C2F74643E3C74643E3C62B5
:100A90003E3C2F623E3C2F74643E3C2F74723E00FD
:100AA0003C74723E3C74643E4D4143204164647228
:100AB0006573733A20003C2F74643E3C74643E3C82
:100AC000623E3C2F623E3C2F74643E3C2F74723E6B
:100AD000003C74723E3C74643E3C666F726D206DE7
:100AE0006574686F643D2267657422206163746970
:100AF0006F6E3D22223E3C703E3C696E70757420E4
:100B0000747970653D227375626D69742220737407
:100B1000796C653D226865696768743A2035307084
:100B200078222076616C75653D2252656672657328
:100B300068223E3C2F703E3C2F666F726D3E3C2F0C
:100B400074643E3C2F74723E3C2F7461626C653E4F
:100B50003C62723E3C666F726D2069643D22666F36
:100B6000726D226E616D653D22666F726D22206D21
:100B70006574686F643D22676574222061637469DF
:100B80006F6E3D22696E6465782E68746D6C223ECE
:100B90003C6669656C647365743E3C6C6567656E44
:100BA000643E4C454420636F6E74726F6C3C2F6CD6
:100BB0006567656E643E3C696E707574207479700B
:100BC000653D227375626D697422207374796C655A
:100BD0003D226865696768743A2035307078222054
:100BE0006E616D653D22746F67676C65222076616A
:100BF0006C75653D224C454430223E266E62737012
:100C0000266E6273703C696E7075742074797065BD
:100C10003D227375626D697422207374796C653D31
:100C2000226865696768743A203530707822206ED2
:100C3000616D653D22746F67676C65222076616C1B
:100C400075653D224C454431223E266E6273702606
:100C50006E6273703C696E70757420747970653D56
:100C6000227375626D697422207374796C653D22FC
:100C70006865696768743A203530707822206E6143
:100C80006D653D22746F67676C65222076616C75B7
:100C9000653D224C454432223E266E627370266EBC
:100CA0006273703C696E70757420747970653D2252
:100CB0007375626D697422207374796C653D226866
:100CC00065696768743A203530707822206E616DEE
:100CD000653D22746F67676C65222076616C75656F
:100CE0003D224C454433223E266E627370266E626E
:100CF00073703C703E003C696E707574207479703E
:100D0000653D227375626D697422207374796C6518
:100D10003D226865696768743A2035307078222012
:100D20006E616D653D22746F67676C652220766128
:100D30006C75653D224C454434223E266E627370CC
:100D4000266E6273703C696E70757420747970657C
:100D50003D227375626D697422207374796C653DF0
:100D6000226865696768743A203530707822206E91
:100D7000616D653D22746F67676C65222076616CDA
:100D800075653D224C454435223E266E62737026C1
:100D90006E6273703C696E70757420747970653D15
:100DA000227375626D697422207374796C653D22BB
:100DB0006865696768743A203530707822206E6102
:100DC0006D653D22746F67676C65222076616C7576
:100DD000653D224C454436223E266E627370266E77
:100DE0006273703C696E70757420747970653D2211
:100DF0007375626D697422207374796C653D226825
:100E000065696768743A203530707822206E616DAC
:100E1000653D22746F67676C65222076616C75652D
:100E20003D224C454437223E266E627370266E6228
:100E300073703C2F6669656C647365743E3C2F6605
:100E40006F726D3E3C2F74643E3C74643E266E624D
:100E500073703B3C2F74643E3C2F74723E3C2F7485
:100E600061626C653E3C2F74643E3C74642077691B
:100E70006474683D22323025223E3C2F74643E3C2F
:100E80002F74723E3C2F7461626C653E3C2F626F22
:100E900064793E3C2F68746D6C3E006364696E6FCC
:100EA00070737578585B000011241FBECFEFDFE32D
:100EB000DEBFCDBF00E00CBF18BE19BE1ABE1BBE00
:100EC00013E3A0E0B0E2EAE3F8EB00E00BBF02C0FE
:100ED00007900D92AE32B107D9F71BBE14E3AEE214
:100EE000B3E301C01D92A732B107E1F70E94284386
:100EF0000C941B5C0C9400009BB78BBFFB01809192
:100F0000CA014093CA017DE970933400E89580934B
:100F1000CA019BBF08952091CF0127FDFCCF9BB74D
:100F20008BBFFB018091CA0123E22093CA010A0111
:100F3000E89511248093CA019BBF0895E091303356
:100F4000F09131330BC0228122FD05C02081318117
:100F50002817390729F00380F481E02D309799F79D
:100F6000CF0108959C01AB01A0913233B09133338E
:100F7000ED91FC91119716968D919C911797B9015F
:100F8000199508959C01AB01A0913233B091333390
:100F90001296ED91FC91139716968D919C9117974F
:100FA000B90119950895A0913233B0913333149655
:100FB000ED91FC911597309739F016968D919C9193
:100FC000179761E070E019950895A0913233B091C0
:100FD00033331496ED91FC911597309739F01696AE
:100FE0008D919C91179760E070E019950895E091BC
:100FF0003233F0913333808983FD0CC008951C9601
:10100000ED91FC911D97309749F01E968D919C9122
:101010001F971995A0913233B091333351968C912B
:101020005197882361F351961C9251970895AF927E
:10103000BF92CF92DF92EF92FF920F931F93CF93C5
:10104000DF937C015B01EA016901289688E090E06A
:10105000C80ED91ECE010E94D614F7018083918359
:101060001282A3821482158216820115110579F06D
:101070000E94D307C701BE010E94C2070E94F70762
:10108000C701B6010E94B2070E94E5070AC0C70166
:10109000BE010E94C2070E94F707C701B6010E9465
:1010A000B207F701808191810E94DA14F7018083F1
:1010B0009183848195810E94DA149C01F7018483D5
:1010C0009583808191818C159D0541F482818130C9
:1010D00029F4838190E08A159B0511F020EF3FEF02
:1010E000C901DF91CF911F910F91FF90EF90DF9099
:1010F000CF90BF90AF900895CF92DF92EF92FF9282
:101100000F931F93CF93DF937C016B01EA01890159
:10111000E0913233F091333320853185211531054B
:1011200031F08285938561E070E0F9011995C7017E
:10113000B601AE01980101E010E00E941708082FE7
:10114000C92FA0913233B09133331896ED91FC91B1
:101150001997309739F01A968D919C911B9760E002
:1011600070E01995802F9C2FDF91CF911F910F91E7
:10117000FF90EF90DF90CF9008954F925F926F9223
:101180007F928F929F92AF92BF92CF92DF92EF9217
:10119000FF920F931F93CF93DF93EC015B014A0102
:1011A000390128010091323310913333C8018A96F6
:1011B00069E070E040E050E020E430E00E947C080C
:1011C0009C01209749F0F80182A993A9A4A9B5A987
:1011D00088839983AA83BB83A114B10451F0F801D9
:1011E00086A997A9A0ADB1ADF50180839183A283B3
:1011F000B3838114910451F0F80182AD93ADA4AD95
:10120000B5ADF40180839183A283B383611471042B
:1012100059F0F801FE9680819181A281B381F3019A
:1012200080839183A283B3834114510451F0F80168
:10123000E159FF4F8081992787FD9095F2018083C6
:101240009183C114D10451F0F801E259FF4F80811C
:10125000992787FD9095F60180839183E114F1042D
:1012600061F0F801EE5BFF4F80819181A281B38133
:10127000F70180839183A283B383C901DF91CF916A
:101280001F910F91FF90EF90DF90CF90BF90AF90A4
:101290009F908F907F906F905F904F9008950F93E5
:1012A000CF93DF93E0913233F0913333009751F0D5
:1012B000EC0188819981AA81BB8182AB93ABA4ABFD
:1012C000B5AB04C012AA13AA14AA15AA6115710518
:1012D00051F0EB0188819981AA81BB8186AB97ABE4
:1012E000A0AFB1AF04C016AA17AA10AE11AE411537
:1012F000510551F0EA0188819981AA81BB8182AFB1
:1013000093AFA4AFB5AF04C012AE13AE14AE15AE1A
:10131000DF01DE962115310559F0E9014881598137
:101320006A817B814D935D936D937C93139705C088
:101330001D921D921D921C921397DF01AE5BBF4F51
:101340000C93CF018A9668E070E044E150E020E021
:1013500030E00E947C08DF91CF910F910895CF92E9
:10136000DF92EF92FF920F931F93CF93DF936C0165
:10137000EB010091323310913333209709F454C0BC
:10138000CB0183709070009729F0862F837024E042
:10139000281B01C020E08AE2E82EF12CE00EF11EAD
:1013A000F80120ABCE010896820F911D0E94D61441
:1013B000F80182A793A782E084A78BE185A716A6F0
:1013C00017A6C70168E070E00E94C207F80180A973
:1013D000C80FD11DC601BE010E94C2078C179D0710
:1013E00031F50E94F707C70168E070E00E94B2077C
:1013F000F80182A593A50E94DA14F80182A793A7A9
:1014000086A597A50E94DA149C01F80186A797A7E4
:1014100082A593A58830910551F484A5833039F4D1
:1014200085A58B3131F003C020E030E002C020EF11
:101430003FEFC901DF91CF911F910F91FF90EF9086
:10144000DF90CF900895AF92BF92CF92DF92EF924C
:10145000FF920F931F93CF93DF935C017B016A018F
:10146000E9018BE593E3809332339093333360E06B
:1014700070E04AEB50E00E94EA16E0913233F091BE
:101480003333E082F182C282D382C483D583068360
:10149000178381E0A816B10419F480898860808BD5
:1014A00080E090E0DF91CF911F910F91FF90EF903E
:1014B000DF90CF90BF90AF9008950F931F93CF937D
:1014C000DF938C01C0913233D0913333CE018A96B1
:1014D00063E270E040E050E024E030E00E947C08ED
:1014E00097FD05C08AA9F801808380E090E0DF9134
:1014F000CF911F910F910895EF92FF920F931F9339
:10150000CF93DF93EC018B01E0913233F0913333D1
:10151000009719F081E082AB01C012AACF018A9630
:101520006FE170E044E050E020E030E00E947C0891
:101530007C01E0913233F0913333C087D187028749
:101540001387C80160E070E0FE011995C701DF91C3
:10155000CF911F910F91FF90EF900895E09132335A
:10156000F091333384879587668777870895E09174
:101570003233F091333381E0818B08950F931F93C1
:10158000CF93DF930F92CDB7DEB700913233109136
:10159000333349830E94DE14DC01CB01F80182ABB6
:1015A00093ABA4ABB5AB498146AB809132339091FC
:1015B00033338A9660E070E048E050E024E030E0A9
:1015C0000E947C080F90DF91CF911F910F91089599
:1015D0006F927F928F929F92AF92BF92CF92DF9243
:1015E000EF92FF920F931F93CF93DF933C017B0108
:1015F0006A014901C0913233D0913333CE018A96CA
:1016000062E070E040E050E024E230E00E947C08BC
:101610005C0197FD3AC08AA990E0A0E0B0E0BC016F
:10162000552744278CA990E0A0E0B0E0482B592B27
:101630006A2B7B2B8BA990E0A0E0B0E0BA2FA92FFA
:10164000982F8827482B592B6A2B7B2BF30140833B
:10165000518362837383E114F10451F0C114D10406
:1016600039F0BE016A5C7F4FC701A6010E94F916DE
:101670008114910451F00115110539F0BE016A5B26
:101680007F4FC401A8010E94F916C501DF91CF91D7
:101690001F910F91FF90EF90DF90CF90BF90AF9090
:1016A0009F908F907F906F900895E0913233F091EA
:1016B0003333828B938B648B758B0895CF92DF923B
:1016C000EF92FF920F931F93CF93DF938C017B01D7
:1016D0006A01C0913233D0913333E296CE0160E09B
:1016E00070E044E250E00E94EA16E0913233F0915B
:1016F0003333E6A2F7A2C0A6D1A60115110531F039
:10170000CE01B80141E250E00E94E71680913233E9
:10171000909133338A9665E270E044E250E020E035
:1017200030E00E947C08DF91CF911F910F91FF90D4
:10173000EF90DF90CF900895AF92BF92CF92DF925B
:10174000EF92FF920F931F93CF93DF938C016B0166
:101750005A01E0903233F0903333E701E296CE0144
:1017600060E070E048E650E00E94EA1601151105BD
:1017700031F0CE01B80141E250E00E94E716C114F9
:10178000D10461F081E0A816B10439F1C6010E94CC
:10179000F01608978833910500F112C0F701EA5658
:1017A000FF4FA08280913233909133338A9663E069
:1017B00070E048E650E020E030E00E947C0802C083
:1017C0008EEF9FEFDF91CF911F910F91FF90EF90E0
:1017D000DF90CF90BF90AF900895C7018A5A9F4F76
:1017E000B6014FE350E00E94F916D8CF8091323312
:1017F000909133338A9664E070E040E050E020E05E
:1018000030E00E947C0808950F931F9300E010E0E1
:101810000E944F091F910F910895CF92DF92EF928E
:10182000FF920F931F9300E010E0EE24FF24CC24DE
:10183000DD240E94BD081F910F91FF90EF90DF9073
:10184000CF9008950F931F938C0180E090E060E0AB
:1018500070E040E050E020E030E00E944F091F912E
:101860000F910895CF92DF92EF92FF920F931F9303
:101870008C0180E090E060E070E040E050E020E02B
:1018800030E0EE24FF24CC24DD240E94BD081F910B
:101890000F91FF90EF90DF90CF900895E091323359
:1018A000F091333382ABCF018A9669E170E044E076
:1018B00050E020E030E00E947C080895E09132334F
:1018C000F0913333868B978B608F718F08950F93D0
:1018D0001F93CF93DF938C01C0913233D091333378
:1018E0000097D9F0CE018A9666E070E040E050E0C3
:1018F00024E330E00E947C0897FF04C02FEF8C3F68
:10190000920769F4BE016E5C7F4FC80146E050E06B
:101910000E94E71680E090E002C08EEF9FEFDF911B
:10192000CF911F910F9108950F931F93CF93DF9342
:10193000EC0100913233109133330097A9F1C801C3
:101940008A9666E070E040E050E024E330E00E94D8
:101950007C0897FD2BC0B801685C7F4FCE01849650
:1019600046E050E00E94E716B801625C7F4FCE016E
:1019700041E250E00E94E716F801EE59FF4F8081E6
:1019800091810E94DA148AA79BA7F801EC59FF4FB6
:10199000808191810E94DA148CA79DA71AA219A2B6
:1019A0001BA280E090E002C08EEF9FEFDF91CF910D
:1019B0001F910F910895CF92DF92EF92FF920F93B4
:1019C0001F93CF93DF930F92CDB7DEB7F82EC09061
:1019D0003233D09033338FE090E069830E944E47DA
:1019E0008C016981009779F1F601F2AA63AB8091CD
:1019F0003233909133338A966BE070E044E050E0EC
:101A000020E030E00E947C087C0197FF04C0C80100
:101A10000E9466471CC0F801808391831382148260
:101A2000E0913033F0913133309731F4009330331B
:101A3000109331330CC0FC01838194810097D9F756
:101A40000383148304C04DEFE42E4FEFF42EC7013F
:101A50000F90DF91CF911F910F91FF90EF90DF904A
:101A6000CF9008950F931F93CF93DF938B01EA01DB
:101A70000E949E07FC01009739F007831087C387F7
:101A8000D48780E090E002C08EEF9FEFDF91CF918E
:101A90001F910F9108950F931F93CF93DF938B01A5
:101AA000EA010E949E07FC01009739F00187128726
:101AB000C587D68780E090E002C08EEF9FEFDF9170
:101AC000CF911F910F910895EF92FF920F931F9363
:101AD000CF93DF93EB017A010091323310913333CE
:101AE0000E94D614F80186AB97AB88819981AA81B0
:101AF000BB8182AB93ABA4ABB5ABC7010E94D6143C
:101B0000F80180AF91AF80913233909133338A9650
:101B10006CE070E048E050E020E030E00E947C089B
:101B2000DF91CF911F910F91FF90EF900895AF92A9
:101B3000BF92CF92DF92FF920F931F93CF93DF93C9
:101B40008C01F62E5A016901C0913233D0913333A2
:101B50000E949E07FC010097C9F0A582B682C38649
:101B6000D4861282C8010E94D6148AAB9BABFCAA11
:101B700080913233909133338A966DE070E044E087
:101B800050E020E030E00E947C0802C08EEF9FEF22
:101B9000DF91CF911F910F91FF90DF90CF90BF9079
:101BA000AF900895CF92DF92EF92FF920F931F9321
:101BB000CF93DF937C01EB016A01009132331091E6
:101BC00033330E949E07009721F1FC011282C70166
:101BD0000E94D614F80186AB97AB88819981AA81BF
:101BE000BB8182AB93ABA4ABB5ABC6010E94D6144C
:101BF000F80180AF91AF80913233909133338A9660
:101C00006EE070E048E050E020E030E00E947C08A8
:101C100002C08EEF9FEFDF91CF911F910F91FF9048
:101C2000EF90DF90CF900895EF92FF920F931F9364
:101C3000CF93DF937C01C0913233D09133338FE067
:101C400090E00E944E478C01009771F1C7010E94FD
:101C5000D6148AAB9BAB80913233909133338A9602
:101C600064E170E044E050E020E030E00E947C0855
:101C7000EC0197FF04C0C8010E94664717C0F80135
:101C80008083918313821482828181608283E091B8
:101C90003033F091313301C0FC018381948100978E
:101CA000D9F70383148302C0CDEFDFEFCE01DF91BC
:101CB000CF911F910F91FF90EF9008950F931F9375
:101CC000CF93DF938C01C0913233D09133330E9494
:101CD000D6148AAB9BAB80913233909133338A9682
:101CE0006FE070E044E050E020E030E00E947C08CB
:101CF0002091303330913133F901C0E0D0E02DC074
:101D0000808191818017910719F5828182FD20C021
:101D1000A0913233B091333350969C91509792FFFB
:101D200003C0846082831BC0209751F4D9011396AD
:101D30008D919C911497809330339093313304C0EC
:101D4000838194818B839C83CF010E94664707C067
:101D500093818481EF01E92FF82F309789F680E095
:101D600090E0DF91CF911F910F9108958F929F92F4
:101D7000AF92BF92CF92DF92EF92FF920F931F9399
:101D8000CF93DF9300D0CDB7DEB74B017A0100913E
:101D90003233109133330E94D614F80182AB93ABE7
:101DA000C7010E94D614F80184AB95ABA0913233E1
:101DB000B09133331896ED91FC911997309739F023
:101DC0001A968D919C911B9761E070E019950E9485
:101DD000D30780913233909133338A9660E170E07B
:101DE00044E050E020E030E000E010E00E941708FE
:101DF0005C0197FD4DC0E816F9060CF445C0C09093
:101E00003233D09033330097C1F10E94F707C601F7
:101E10008A9668E070E00E94B2078C01F60182A504
:101E200093A50E94DA14F60182A793A70830110542
:101E300039F524A5243021F525A52B3109F520A954
:101E400068EFE62E6FEFF62EE21AF108E80EF91EA3
:101E5000EA14FB04A9F4C401B7010E94B2078C0183
:101E60008E159F0569F4F60160A9662359F0CE012D
:101E7000019670E00E94B20705C000E010E002C0C9
:101E800000EF1FEF580104C050EFA52E5FEFB52EF5
:101E90000E94E507A0913233B09133331896ED914B
:101EA000FC911997309739F01A968D919C911B9758
:101EB00060E070E01995C5012396CDBFDEBFDF91CC
:101EC000CF911F910F91FF90EF90DF90CF90BF9037
:101ED000AF909F908F900895CF92DF92EF92FF92F4
:101EE0000F931F93CF93DF936B017A01C09132332D
:101EF000D09133330E94D6148AAB9BABC7010E94AA
:101F0000D6148CAB9DABA0913233B091333318967D
:101F1000ED91FC911997309739F01A968D919C911B
:101F20001B9761E070E019950E94D30780913233CE
:101F3000909133338A9661E170E044E050E020E014
:101F400030E000E010E00E941708EC0197FD0BC0A4
:101F5000E816F90634F0C601BE010E94AF09EC0193
:101F600002C0C0EFDFEF0E94E507A0913233B091CD
:101F700033331896ED91FC911997309739F01A96F2
:101F80008D919C911B9760E070E01995CE01DF91D7
:101F9000CF911F910F91FF90EF90DF90CF90089518
:101FA000AF92BF92CF92DF92EF92FF920F931F9367
:101FB000CF93DF935B016A01E9017801009132332D
:101FC000109133330E94D614F80186AB97ABC6014B
:101FD0000E94D614F80180AF91AF88819981AA81BF
:101FE000BB8182AB93ABA4ABB5ABC7010E94D61447
:101FF000F80182AF93AFA0913233B091333318968A
:10200000ED91FC911997309739F01A968D919C912A
:102010001B9761E070E019950E94D30780913233DD
:10202000909133338A9662E170E04CE050E020E01A
:1020300030E000E010E00E941708EC0197FD0BC0B3
:10204000C816D90634F0C501BE010E94AF09EC01E3
:1020500002C0C0EFDFEF0E94E507A0913233B091DC
:1020600033331896ED91FC911997309739F01A9601
:102070008D919C911B9760E070E01995CE01DF91E6
:10208000CF911F910F91FF90EF90DF90CF90BF9075
:10209000AF9008950F931F93CF93DF938B01C0915F
:1020A0003233D09133330E94D6148AAB9BAB8091EC
:1020B0003233909133338A9665E170E044E050E02A
:1020C00024E030E00E947C0897FD09C04AA95BA982
:1020D0006CA97DA9F8014083518362837383DF91EA
:1020E000CF911F910F910895CF92DF92EF92FF92BF
:1020F0000F931F93CF93DF93EC017B016A01009153
:10210000323310913333009751F10E94F01680382A
:10211000910528F5E0913233F0913333828D938D20
:10212000009701F5C801C296BE010E940217809176
:102130003233909133338A966AE070E040E850E0A1
:1021400020E030E00E947C0897FD0EC0E091323321
:10215000F0913333E28EF38EC48ED58E05C08EEFB0
:102160009FEF02C082EF9FEFDF91CF911F910F9100
:10217000FF90EF90DF90CF900895CF92DF92EF9293
:10218000FF920F931F93CF93DF93CDB7DEB72C97BA
:10219000CDBFDEBF8091323390913333009709F485
:1021A0005DC28A9661E070E040E050E020E030E0FF
:1021B0000E947C08009709F451C2809132339091BB
:1021C00033338A9665E070E040E050E020E030E094
:1021D0000E947C08A0913233B09133330097B1F460
:1021E0005296ED91FC915397309741F150968C9116
:1021F000509780FD23C0816050968C9350975496E1
:102200008D919C91559761E070E017C097FF16C0C3
:102210005296ED91FC915397309781F050968C91A6
:10222000509780FF0BC08E7F50968C93509754969A
:102230008D919C91559760E070E01995E091323353
:10224000F091333386A197A1009709F451C08F0113
:10225000045A1F4FAEE5EA2EF12CEE0EFF1EB2E33C
:10226000CB2ED12CCE0EDF1E8091323390913333A2
:102270008A9666E270E040E050E020E330E00E94A1
:102280007C080097B1F4A0913233B0913333969625
:10229000ED91FC91979798968D919C91999760E01C
:1022A00070E01995E0913233F091333316A217A202
:1022B0001FC018161906E4F4D8018D919C910E9454
:1022C000DA14F80180839183D7018D919C910E944B
:1022D000DA14F70180839183E0913233F091333344
:1022E00026A137A180A591A5B601F9011995BCCF0A
:1022F000CE01099660E070E040E050E020E030E080
:102300008E010F5F1F4FE5E0EE2EF12CEC0EFD1E4F
:10231000F3E0CF2ED12CCC0EDD1E0E94BD089C0117
:1023200089819A81009739F4E0913233F091333307
:1023300040894D7F408BE0913233F091333321154A
:102340003105A1F4009739F1268937892115310526
:1023500011F1808981FD1FC08260808B808D918DFD
:10236000BE01675F7F4FF901199515C037FF3AC06D
:102370000097C1F1268937892115310599F18089A6
:1023800081FF30C08D7F808B808D918D60E070E00B
:10239000F901199527C0A0913233B09133335A9681
:1023A000ED91FC915B973097E9F08B819C810097D0
:1023B00041F45C968D919C915D97BE016B5F7F4F60
:1023C0000AC02FEF8F3F920769F45C968D919C9124
:1023D0005D9760E070E01995E0913233F09133330E
:1023E000128E138EE0913233F0913333268D378D78
:1023F00021153105C1F0DF01AA5BBF4F4D915C9102
:1024000011974115510579F0BF01685B7F4F80A19D
:1024100091A1F9011995E0913233F0913333168E81
:10242000178E10A211A20091323310913333D801CC
:1024300050968C91509784FF32C092968D919C91CA
:102440009397009761F1C8018A9664E270E040E0DA
:1024500050E024E030E00E947C0897FD03C0F801C2
:1024600082A901C080E0A0913233B091333380FF64
:102470000AC09296ED91FC91939794968D919C91C0
:10248000959761E00BC081FF0AC09296ED91FC9197
:10249000939794968D919C91959760E01995E09112
:1024A0003233F091333380898460808B00913033F4
:1024B0001091313393C0D8018D919C910E94D61414
:1024C000F70182AB93AB80913233909133338A968C
:1024D00063E170E044E050E024E030E00E947C08DA
:1024E000AC0197FD22C0D701D2968C91D297813052
:1024F000D1F4F801928190FD42C00780F085E02D73
:102500003097E9F1892F81608D7FD80112968C93E5
:1025100012976D917C9111971B968D919C911C97B0
:1025200041E050E057C08430B9F4F801828181FD68
:1025300025C00780F085E02D309701F18E7F826005
:10254000D80112968C9312976D917C9111971B96DE
:102550008D919C911C973CC0833089F4D8011596CD
:10256000ED91FC911697309751F06D917C911197F8
:102570001B968D919C911C9719952DC084E0141683
:1025800015067CF4D8011996ED91FC911A973097B5
:1025900041F06D917C9111971D968D919C911E97A4
:1025A00019C08823C1F4F801828180FF14C001841E
:1025B000F285E02D309779F08E7FD80112968C93BA
:1025C00012976D917C9111971D968D919C911E97FC
:1025D00040E050E01995F80103811481E090323316
:1025E000F09033330115110509F065CFD7015096EE
:1025F0008C9150978B7F50968C935097E09130330D
:10260000F091313300E010E027C0828182FF1FC0CB
:102610000115110569F4A0913033B091313313964F
:102620008D919C911497809330339093313307C0F0
:1026300083819481D80113968D939C931497C380C2
:10264000E480CF010E946647EC2DFE2D05C09381EA
:1026500084818F01E92FF82F3097B9F680E090E060
:102660002C96CDBFDEBFDF91CF911F910F91FF90D0
:10267000EF90DF90CF900895E0913233F0913333B3
:1026800082ABCF018A9667E270E044E050E020E040
:1026900030E00E947C0808959C01E0913233F09173
:1026A0003333868D978D009779F4268F378F60A30B
:1026B00071A3CF018A9668E270E040E050E020E02C
:1026C00030E00E947C0808958EEF9FEF0895BC01D2
:1026D0008091323390913333C29646E250E00E94AB
:1026E000E71680913233909133338A9669E270E035
:1026F00048E250E020E030E00E947C080895E0913C
:102700003233F091333382ABCF018A9666E170E0C9
:1027100044E050E020E030E00E947C0808950F93F0
:102720001F93CF93DF938C01C0913233D091333319
:10273000CE018A966AE170E040E050E024E030E0AB
:102740000E947C0897FD03C02AA9F8012083DF912D
:10275000CF911F910F910895E0913233F09133336F
:1027600082ABCF018A9667E170E044E050E020E060
:1027700030E00E947C08089586EF9FEF0895E09175
:102780003233F091333321E0009709F420E022AB9B
:10279000CF018A966EE170E044E050E020E030E046
:1027A0000E947C0808958F929F92AF92BF92CF9221
:1027B000DF92EF92FF920F931F93CF93DF93F82E48
:1027C0004A015B01C901B801C0913233D091333362
:1027D0000E94DE14DC01CB018AAB9BABACABBDAB82
:1027E000C501B4010E94DE14DC01CB018EAB9FABAE
:1027F000A8AFB9AFC6010E94D6148AAF9BAFFCAE9A
:10280000EDAE80913233909133338A966DE170E072
:102810004FE050E020E030E00E947C08DF91CF9153
:102820001F910F91FF90EF90DF90CF90BF90AF90EE
:102830009F908F900895AF92BF92DF92EF92FF9298
:102840000F931F93CF93DF93D82EEB015A01790199
:102850000091323310913333C801C29660E070E0CA
:1028600048E850E00E94EA16209749F08881998153
:10287000AA81BB81F80182AB93ABA4ABB5ABC50118
:102880000E94D614F80186AB97ABD0AEE114F104E8
:1028900079F0C7010E94F0168F37910500F5C70146
:1028A0000E94F016AC01C801CA96B7010E94E71653
:1028B00080913233909133338A966CE170E048E82E
:1028C00050E020E030E00E947C08009751F4E09155
:1028D0003233F091333320892061208B02C08EEF98
:1028E0009FEFDF91CF911F910F91FF90EF90DF90BD
:1028F000BF90AF900895E0913233F091333382A3CB
:1029000093A364A375A380E090E00895E09132332F
:10291000F091333321E0009709F420E022ABCF019E
:102920008A9660E270E044E050E020E030E00E94EF
:102930007C080895CF93DF93C0913233D091333325
:102940000E94DE14DC01CB018AAB9BABACABBDAB10
:1029500080913233909133338A9661E270E044E0A3
:1029600050E020E030E00E947C08DF91CF91089594
:10297000CF93DF93C0913233D09133330E94DE1472
:10298000DC01CB018AAB9BABACABBDAB80913233EE
:10299000909133338A9662E270E044E050E020E0A8
:1029A00030E00E947C08DF91CF9108959827892715
:1029B0009827089598278927982708950F931F939C
:1029C000DC01CB010B2F112722273327782F662715
:1029D00055274427042B152B262B372B4427582FFC
:1029E000692F7A2F407050707070042B152B262B96
:1029F000372B892F9A2FAB2FBB278070A070B07018
:102A0000082B192B2A2B3B2BB801C9011F910F91C1
:102A100008950E94DE1408952F923F924F925F9284
:102A20006F927F928F929F92AF92BF92CF92DF92DE
:102A3000EF92FF920F931F93CF93DF93CDB7DEB743
:102A40006497CDBFDEBFFC016B8B7C8B00811127AF
:102A500007FD10959E01235F3F4F298B3A8B7E0126
:102A60000894E11CF11C802F80538A3008F03EC18D
:102A700000331105C1F40181112707FD10950837B6
:102A8000110541F00835110529F0319628E0622E34
:102A9000712C0CC00281112707FD1095329690E130
:102AA000692E712C03C08AE0682E712C6F0140E002
:102AB00050E0BA011301442437FC4094542C902F69
:102AC000802F80538A30A0F4CB01BA01A20191017A
:102AD0000E94DC504B015C01C801C097AC01662725
:102AE00057FD6095762F480D591D6A1D7B1D2AC024
:102AF000B0E16B16710489F5802F8156863020F085
:102B0000202F2154263048F54A015B01B4E0880C9F
:102B1000991CAA1CBB1CBA95D1F7065F1F4F8A31BE
:102B200018F481E690E002C081E490E0F801E81B2F
:102B3000F90BAF01662757FD6095762F4829592973
:102B40006A297B29D60111960C911197112707FD4F
:102B500010950894C11CD11CB2CFE42F352F0E3232
:102B60001105F1F449895A89E416F50609F4BEC045
:102B7000D701EC9311963C93119712966C93129790
:102B800013967C93E4E0F0E0EE0EFF1EF601319622
:102B9000D60111960C911197112707FD109563CF5F
:102BA00001151105C1F0903208F4A0C007FD9EC0C8
:102BB0000032110581F00C30110569F00A30110561
:102BC00051F00D30110539F00930110521F00B30AD
:102BD000110509F08BC0CE010196E81AF90AF594A7
:102BE000E794F594E7940894E11CF11CB2E0EB162D
:102BF000F10499F0E3E0EE16F1042CF4E114F10491
:102C000009F474C062C0F3E0EF16F104E1F024E0CF
:102C1000E216F10409F059C02FC0403030E05307EC
:102C200030E0630731E0730708F060C089819A8162
:102C3000AB81BC81B82FAA2799278827482B592B0D
:102C40006A2B7B2B42C0403080E0580781E0680748
:102C500080E0780708F04AC00D811E812F813885F9
:102C600098011127002789819A81AB81BC81B82FF7
:102C7000AA279927882721C04F3F51056105710573
:102C800009F0A0F50D811E812F813885980111274B
:102C9000002789819A81AB81BC81B82FAA27992707
:102CA0008827082B192B2A2B3B2B89859A85AB85E6
:102CB000BC85BA2FA92F982F8827082B192B2A2BD0
:102CC0003B2B402B512B622B732BAB89BC8910976C
:102CD00081F0CB01BA010E94DE14DC01CB01EB894B
:102CE000FC8980839183A283B38303C080E090E05A
:102CF00002C081E090E06496CDBFDEBFDF91CF914E
:102D00001F910F91FF90EF90DF90CF90BF90AF9009
:102D10009F908F907F906F905F904F903F902F90FB
:102D200008950F931F93CF93DF93CDB7DEB7279707
:102D3000CDBFDEBFFC0180819181A281B3818C83F4
:102D40009D83AE83BF83AE014C5F5F4F20E0E4E321
:102D5000F3E31AE00EE2DA018C9130E0612F0E9479
:102D6000FB50A1E0B0E0AC0FBD1FA30FB11D905D03
:102D70009C933F5F882391F7632FDA011D92AD0189
:102D8000CF010BC03150A1E0B0E0AC0FBD1FA30FCD
:102D9000B11D7C91DC017D93CD01332399F7DF01D7
:102DA000A60FB11DFD0101932F5F2430A1F61C92E7
:102DB00084E393E32796CDBFDEBFDF91CF911F91D0
:102DC0000F9108950E94484780E090E008950E9486
:102DD000E35408950E94FE5408950E94EC5408950F
:102DE000FC0101900020E9F73197E81BF90BCF01B6
:102DF00008950E94645508950E94565508950E94B2
:102E00002E5508950E9437550895EF92FF920F9323
:102E10001F93CF93DF937C01EB01CB0101960E94BE
:102E20004B478C01009739F0B701AE010E94645501
:102E3000C00FD11F1882C801DF91CF911F910F9150
:102E4000FF90EF900895DC010D900020E9F7BD019F
:102E500061507040681B790B0E94051708950E940D
:102E6000185508950E94D65408950E947A530895E3
:102E70000E94235508950E94735508950E94055598
:102E800008950E947E5508950E94D15408950E948D
:102E90003E550895CF92DF92EF92FF920F931F93CA
:102EA000CF93DF937C01D62EC72EDC010D9000203E
:102EB000E9F78D0101501040081B190BE62FF72F81
:102EC000EF0109900020E9F72197CE1BDF0B0DC021
:102ED000C7016D2D7C2DAE010E943E55009751F02B
:102EE0000894E11CF11C015010400C171D0780F7DD
:102EF000EE24FF24C701DF91CF911F910F91FF9026
:102F0000EF90DF90CF900895CF93DF93CDB7DEB7EA
:102F10009E01245F3F4F8E819F81688579854A8518
:102F20005B850E941256DF91CF9108950E94125640
:102F30000895CF92DF92EF92FF920F931F93CF935A
:102F4000DF93CDB7DEB7CC84DD848E01025F1F4FE7
:102F500080EA90E00E944B477C01009771F060EAA4
:102F600070E0A60198010E9412568C0197FD02C0E4
:102F7000670107C0C7010E94664786010DC00E9415
:102F8000A746F60181916F018823C9F7C7010E9406
:102F9000664709C00E94A746F80181918F018823E6
:102FA000C9F70FEF1FEFC801DF91CF911F910F916C
:102FB000FF90EF90DF90CF9008958F929F92AF9205
:102FC000BF92CF92DF92EF92FF920F931F93CF9316
:102FD000DF938C010097B9F1DC011C968D919C91D7
:102FE0001D970E946647D8011296ED91FC911397A8
:102FF000E080F18022E0C22ED12CC00ED11EA12C87
:1030000031E0B32E812C42E0942E17C0C281D381CF
:10301000A081B1811296CD93DC931397A883B983D5
:10302000A082B18282829382CF0106970E94664776
:10303000F70190818181E92EF82EEC15FD0531F71D
:10304000C8010E946647DF91CF911F910F91FF90B9
:10305000EF90DF90CF90BF90AF909F908F900895AA
:10306000CF92DF92EF92FF920F931F93CF93DF9354
:10307000EC016B017A0189018AE090E00E944E47E1
:10308000FC010097C9F0C082D182E282F3820483FE
:1030900015839C012A5F3F4FAC81BD812C833D830A
:1030A000CE01029686839783A087B1872D933C93A8
:1030B000119780E090E002C08DEF9FEFDF91CF91FC
:1030C0001F910F91FF90EF90DF90CF90089520E037
:1030D00030E00E9430180895FC0162AB73AB44AB42
:1030E00055AB0895FC01808191810895FC0184898C
:1030F0009589887090700895FC0180A991A9089520
:10310000CF92DF92EF92FF920F931F93CF93DF93B3
:10311000CDB7DEB7CC84DD848E01005F1F4F80E524
:1031200090E00E944B477C010097F1F060E570E071
:103130004E855F8598010E949617AC0197FF04C0E9
:10314000C7010E94664710C0D6011896ED91FC9108
:1031500019971A968D919C911B97B70119958C011F
:10316000C7010E94664702C00DEF1FEFC801DF9143
:10317000CF911F910F91FF90EF90DF90CF90089526
:103180004F925F926F927F928F929F92AF92BF9277
:10319000CF92DF92EF92FF920F931F93CF93DF9323
:1031A000CDB7DEB76497CDBFDEBF7C01DC011296E0
:1031B0000D911C91139752E0A52EB12CA80EB91EAB
:1031C0006E010894C11CD11C64E1862E912C71E023
:1031D000672E70E2772EE7E04E2EE0E25E2E55C0BD
:1031E000D8011697ED91FC911197208131811496A9
:1031F0008D919C911597009711F480E090E2EDB7C6
:10320000FEB73A97EDBFFEBF3196ADB7BEB7119688
:10321000CD92DC9212978282938264827582268399
:103220003783808791870E948417F8013697019031
:10323000F081E02D84819581EDB7FEB73A96EDBF20
:10324000FEBF009711F480E090E22DB73EB7285002
:1032500030402DBF3EBFEDB7FEB73196ADB7BEB71C
:103260001196ED92FC92129742825382C482D582CB
:10327000868397830E948018F801008111812DB701
:103280003EB7285F3F4F2DBF3EBF0A151B0509F013
:10329000A7CF6496CDBFDEBFDF91CF911F910F9175
:1032A000FF90EF90DF90CF90BF90AF909F908F9066
:1032B0007F906F905F904F900895EF92FF920F93E1
:1032C0001F93CF93DF938C01EB01DC0154968C911B
:1032D000549783FF21C077FD03C082E190E202C0D2
:1032E00085E190E2EDB7FEB73897EDBFFEBF3196AE
:1032F000ADB7BEB711960D931C93129729E130E23A
:103300002283338384839583C683D7830E94801866
:10331000EDB7FEB738962CC077FD05C0A2E1EA2EC6
:10332000A0E2FA2E04C0F5E1EF2EF0E2FF2ECE016E
:103330000E948E1F2DB73EB72A5030402DBF3EBF92
:10334000EDB7FEB73196ADB7BEB711960D931C938E
:10335000129721E230E222833383E482F582C6832E
:10336000D783808791870E948018EDB7FEB73A9681
:10337000EDBFFEBFDF91CF911F910F91FF90EF90B6
:1033800008952F923F924F925F926F927F928F9209
:103390009F92AF92BF92CF92DF92EF92FF920F93E4
:1033A0001F93CF93DF93CDB7DEB7C455D040CDBFC9
:1033B000DEBF5C012901DC0154968C91549783FD9A
:1033C00027C0EDB7FEB73897EDBFFEBF3196ADB75A
:1033D000BEB71196AD92BC92129782E390E28283BF
:1033E0009383648375832683378364964FAF649792
:1033F00065965FAF65970E948018EDB7FEB7389667
:10340000EDBFFEBF65965FAD659764964FAD64975F
:103410004A01CC24DD249E012F5A3F4F63962EAFE4
:103420003FAF63971E010894211C311CAFC08DB7BC
:103430009EB708978DBF9EBFEDB7FEB73196ADB76B
:10344000BEB711962D923C92129720E530E0228370
:1034500033838AE490E284839583C682D7820E9474
:1034600084173101680E791EADB7BEB71896ADBF8F
:10347000BEBF730100E010E0C8018C0D9D1D8415D6
:1034800095055CF5EDB7FEB73897EDBFFEBFADB75C
:10349000BEB71196E182F28263968EAD9FAD6397BF
:1034A0008E199F0912968D939C93139721E530E214
:1034B00014962D933C931597F401E00FF11F808132
:1034C00016968C93169717961C920E9484178DB7A8
:1034D0009EB708968DBF9EBF05C0C7016EE270E221
:1034E0000E940217A3E0B0E0EA0EFB1E0F5F1F4F21
:1034F0000031110509F6D301D09620E030E0C90172
:103500008C0D9D1D841595057CF4F401E20FF31FCD
:103510004081542F5052CD010196503610F44C93F7
:1035200002C0EEE2EC93DC012F5F3F4F203131050A
:1035300031F71C92D50154968C91549783FF03C0A8
:1035400080E090E202C08EE290E2EDB7FEB73897DD
:10355000EDBFFEBF3196ADB7BEB71196AD92BC922E
:10356000129727E530E22283338384839583268272
:1035700037820E94801880E190E0C80ED91E880E24
:10358000991EADB7BEB71896ADBFBEBFC414D50463
:103590000CF44DCFCC5ADF4FCDBFDEBFDF91CF91C2
:1035A0001F910F91FF90EF90DF90CF90BF90AF9061
:1035B0009F908F907F906F905F904F903F902F9053
:1035C00008952F923F924F925F926F927F928F92C7
:1035D0009F92AF92BF92CF92DF92EF92FF920F93A2
:1035E0001F93CF93DF9300D0CDB7DEB78A839B8341
:1035F000DC0152968D919C9153970097D9F150968A
:103600008D919C9151978F3491052CF052961D927B
:103610001C9253973EC26E3679F0623719F06C35C2
:10362000F9F415C0AA81BB811C96ED91FC911D9700
:10363000E80FF91F8DE009C0AA81BB811C96ED91AE
:10364000FC911D97E80FF91F8AE0808309C0AA81C9
:10365000BB811C96ED91FC911D97E80FF91F6083CB
:10366000EA81FB81808991890196808B918B128AF6
:10367000138A0FC26A3009F43FC06B3024F46830FB
:1036800009F0C0C113C06D30B9F16C3509F0BAC191
:10369000AA81BB8154968C91549782FF07C081E028
:1036A00090E052968D939C935397F3C1EA81FB81EE
:1036B00080899189009709F4ECC1848981FD14C047
:1036C00000D00F92ADB7BEB71196ED93FC93129751
:1036D0008EE590E213968D939C9314970E94801828
:1036E0000F900F900F900F90EA81FB818089918954
:1036F0000197808B918BCDC1AA81BB811C96ED91E6
:10370000FC911D9750968D919C915197E80FF91F50
:10371000108254968C91549781FD10C000D00F9266
:10372000EDB7FEB7A183B28382E690E283839483F0
:103730000E9480180F900F900F900F90AA81BB816C
:103740001C968D919C911D9756961D921C92579791
:1037500020E030E258962D933C9359975A962D933A
:103760003C935B9719C0EA81FB8186899789FC01AC
:103770003C96EE0FFF1F4A815B81E40FF51F20830B
:1037800031830196DA0156968D939C9357978C302E
:10379000910549F080E090E065E670E20E944417F0
:1037A0009C01009701F7EA81FB81E08CF18C428C4F
:1037B000538CC7010E94F016009709F4B5C0AA8186
:1037C000BB811296CD90DC901397662477248824D1
:1037D000992492E0292E312C2A0E3B1E48C08601E6
:1037E00006501040D801ED91FC9180819181B70184
:1037F0000E94FF16009751F4F8018481958100978B
:1038000029F0B2010E94FF160097D1F18AEFA82E8D
:103810008FEFB82EAC0CBD1CD501ED91FC918081D1
:103820009181B7010E94FF16009729F4F501848168
:103830009581009729F1D501ED91FC91A080B1808F
:10384000C7010E94F016AC01C501B7010E94FC1629
:10385000009721F48114910419F405C0840103C078
:10386000B1E06B2E712CF601C080D1804801C214EA
:10387000D30409F0B4CF6114710409F055C0840178
:103880000115110509F450C0D80112968D919C9133
:103890001397EA81FB8180839183828D938D0097BA
:1038A00059F114966D917C9115976115710521F16F
:1038B0000E94FF16009701F5D80114968D919C91F6
:1038C0001597EA81FB8180AB91AB808D918D828FC2
:1038D000938F6689778961507040668B778BED9105
:1038E000FC9111974A815B81465E5F4F0280F381B4
:1038F000E02D8A819B8116C0AA81BB81D0961D9242
:103900001C92D197D801ED91FC91AA81BB8156966A
:103910006D917C915797AD01485E5F4F0280F381B6
:10392000E02DCD01199544C0AA81BB81D296ED91BD
:10393000FC91D397309741F0D4968D919C91D59777
:103940008D939C931197E3CFEA81FB81808D918DBC
:103950000E94F016009761F1AA81BB8154968C9168
:10396000549783FF06C0CD0169EE7FEF0E945D1979
:103970001FC000D000D0EDB7FEB731964A815B8101
:10398000ADB7BEB711964D935C93129787E690E260
:1039900082839383DA0158968D919C915997848301
:1039A00095830E948018EDB7FEB73696EDBFFEBF37
:1039B000AA81BB8150961D921C92519754968C916E
:1039C000549780FD66C000D000D0EDB7FEB73196A9
:1039D000AD01ADB7BEB711964D935C9312978EE7CC
:1039E00090E282839383DA0116968D919C911797CA
:1039F000848395830E948018EDB7FEB73696EDBF9D
:103A0000FEBF47C0AA81BB8150968D919C91519772
:103A10008F349105F4F5862F80528F35D0F554966A
:103A20008C91549781FD1FC000D000D0EDB7FEB738
:103A30003196AD01ADB7BEB711964D935C93129719
:103A400082E890E282839383862F992787FD909561
:103A50008483958369830E9480188DB79EB70696EC
:103A60008DBF9EBF6981AA81BB811C96ED91FC919F
:103A70001D9750968D919C915197E80FF91F608387
:103A800050968D919C915197019650968D939C9351
:103A900051972396CDBFDEBFDF91CF911F910F913C
:103AA000FF90EF90DF90CF90BF90AF909F908F905E
:103AB0007F906F905F904F903F902F900895CF929E
:103AC000DF92EF92FF920F931F93CF93DF936C01DE
:103AD0007A018B01C0E0D0E007C0F80161918F014D
:103AE000C6010E94E11A2196CE15DF05B4F3C70185
:103AF000DF91CF911F910F91FF90EF90DF90CF90CA
:103B00000895AF92BF92CF92DF92EF92FF920F9300
:103B10001F93CF93DF93EC016B015A01F22EE32E3A
:103B20006115710509F45DC023FD5BC086E390E07B
:103B30000E944B478C01009709F455C060E070E08B
:103B400046E350E00E94EA16209711F4C5E8D0E25F
:103B5000D8011696CD93DC93179780E590E01E96DA
:103B60008D939C931F970E944B47F80184879587FC
:103B7000009721F4C8010E94DD1733C046855785A0
:103B800060E070E00E94EA16F801F48AE58AC086D7
:103B9000D186A286B386C8010296828393838483EA
:103BA0009583F0FC20C000D000D0EDB7FEB7319671
:103BB000ADB7BEB711960D931C9312978EE790E2A6
:103BC00082839383D80116968D919C911797848355
:103BD00095830E948018EDB7FEB73696EDBFFEBF05
:103BE00002C000E010E0C801DF91CF911F910F915A
:103BF000FF90EF90DF90CF90BF90AF9008952F92FD
:103C00003F924F925F926F927F928F929F92AF926C
:103C1000BF92CF92DF92EF92FF920F931F93CF93B9
:103C2000DF930F920F92CDB7DEB74C0181E090E0A9
:103C300069837A830E944E478C0169817A8100975B
:103C400009F44EC07B01CC24DD24240108944108F2
:103C5000510842C051E0A52EB12CC414D50414F073
:103C6000AA24BB24C8010E94F0161C013701F701E9
:103C7000808191810E94F016B5016F5F7F4F620DC8
:103C8000731D680F791FC8010E9463471C010097CC
:103C900031F4C8010E94664700E010E021C00E9494
:103CA000F01622E030E0E20EF31EF3016081718134
:103CB000820D931D0E940217A114B10449F0C101A5
:103CC0000E94F016820D931D65E670E20E940217B5
:103CD0000894C11CD11C8101C814D9040CF4BACFBA
:103CE000C8010F900F90DF91CF911F910F91FF901E
:103CF000EF90DF90CF90BF90AF909F908F907F908C
:103D00006F905F904F903F902F9008953F924F9209
:103D10005F926F927F928F929F92AF92BF92CF925B
:103D2000DF92EF92FF920F931F93CF93DF93CDB764
:103D3000DEB7C455D040CDBFDEBF4A0100D000D0B1
:103D4000EDB7FEB7319623EA30E2ADB7BEB71196B4
:103D50002D933C9312978283938344835583649677
:103D60006FAF649765967FAF65970E9499176496C9
:103D70006FAD6497A62E65967FAD6597B72EEDB7AC
:103D8000FEB73696EDBFFEBFCC24DD24CE018F5AA0
:103D90009F4F63968EAF9FAF63972E010894411C8F
:103DA000511C6EE2362EA0C0ADB7BEB71897ADBF9E
:103DB000BEBFEDB7FEB7319611964D925C92129749
:103DC00080E590E082839383ABEBB0E2A483B5837C
:103DD000C682D7820E9484173201680E791EEDB721
:103DE000FEB73896EDBFFEBF730100E010E0C801DA
:103DF0008C0D9D1D881599056CF58DB79EB708979C
:103E00008DBF9EBFADB7BEB71196EDB7FEB7E182CD
:103E1000F28263968EAD9FAD63978E199F091296BD
:103E20008D939C93139782EC90E214968D939C93C0
:103E30001597F501E00FF11F808116968C93169768
:103E400017961C920E948417ADB7BEB71896ADBFE7
:103E5000BEBF05C0C70168EC70E20E940217E3E034
:103E6000F0E0EE0EFF1E0F5F1F4F0031110509F04D
:103E7000BECF8301005D1F4FC8016CEC70E20E9451
:103E8000021740E050E0CA018C0D9D1D8815990570
:103E900074F4F501E40FF51F2081C801019620326A
:103EA0001CF0D8012C9302C0F80130828C014F5FC6
:103EB0005F4F4031510539F7D8011C9200D00F9265
:103EC0008FEC90E2EDB7FEB78183928343825482F8
:103ED0000E949917A0E1B0E0CA0EDB1EAA0EBB1E1D
:103EE0000F900F900F900F90C814D9040CF45CCF72
:103EF000CC5ADF4FCDBFDEBFDF91CF911F910F9125
:103F0000FF90EF90DF90CF90BF90AF909F908F90F9
:103F10007F906F905F904F903F900895FC0197FFC6
:103F20000BC07696E631F10550F4EE0FFF1FED5F02
:103F3000FD4C80819181089587ED90E208958FED89
:103F400090E208958EE090E00E944E47FC0180933D
:103F5000483390934933009761F08083F1838283E3
:103F6000F3838085918582608087918780E090E0EF
:103F700008958DEF9FEF08958EE090E00E944E47E8
:103F80000895CF93DF93DC01009779F114968C911B
:103F9000149781FF27C0C0914833D0914933EC81F9
:103FA000FD81CD010A96E817F90721F480819181FE
:103FB0008C839D831C96ED91FC911D971A96CD9153
:103FC000DC911B97EA83FB83C083D18380E091E07F
:103FD0001A968D939C931B9780E092E01C968D938C
:103FE0009C931D97CD010E946647DF91CF91089564
:103FF0000F931F93CF93DF93DC0114968D919C91C7
:1040000015978B7F14968D939C9315972D933C93C6
:10401000119712960D931C931397C0914833D0912A
:1040200049332E813F8116962D933C93179718960E
:104030006D937C9319974115510529F08160149671
:104040008D939C93159714962D913C91159721FD76
:1040500010C0CD010A96EA81FB818A839B831A9660
:10406000CD93DC931B971C96ED93FC931D97808357
:104070009183226014962D933C931597DF91CF91F5
:104080001F910F910895CF93DF93EC012C813D8117
:1040900021FF27C0A0914833B09149331496ED9188
:1040A000FC9115970A96E817F90731F48081918100
:1040B00014968D939C931597EC85FD85AA85BB85F9
:1040C0001296ED93FC931397A083B18380E091E067
:1040D0008A879B8780E092E08C879D872D7F2C8349
:1040E0003D83DF91CF910895FC0184818270089512
:1040F000AF92BF92CF92DF92EF92FF920F931F93F6
:10410000CF93DF937C016B015A0189010E94BC1F90
:10411000EC01009729F0B701A60195010E94F81F54
:10412000CE01DF91CF911F910F91FF90EF90DF9023
:10413000CF90BF90AF9008950E94C11F08950F9334
:104140001F93FC0144815581417050702081318161
:10415000028113810E94F81F1F910F910895E09131
:104160004833F0914933868197810895E09148332F
:10417000F0914933309731F026813781280F391F6C
:104180002683378308956817790728F480959095DA
:10419000860F971F08959B01281B390BC9010895AD
:1041A000CF93DF93EA01209719F08617970739F02C
:1041B0000E94C32021E030E08C179D0710F420E01E
:1041C00030E0C901DF91CF910895EF92FF920F93F4
:1041D0001F93CF93DF938C01C0914833D091493323
:1041E000EE80FF806E817F81C701A8010E94D020F0
:1041F0000097C1F3DF91CF911F910F91FF90EF9046
:1042000008954F925F926F927F928F929F92AF929A
:10421000BF92CF92DF92EF92FF920F931F93CF93B3
:10422000DF930F92CDB7DEB7E0914833F091493379
:104230008085918581FF05C08D7F8087918721E0F2
:1042400001C020E0808591858160808791876080B2
:104250007180D3018D919C91119784839583A12CBA
:1042600031E0B32E812C42E0942E54C066817781D8
:1042700086EFC82E8FEFD82EC60CD71CD601189605
:104280004D915C91199716968D919C911797298362
:104290000E94D0202981009789F1F60184819581BF
:1042A00080FF08C0D80116968D919C911797868340
:1042B000978316C0F301A281B38120813181F90176
:1042C000A283B3832D933C93D301AD92BC921197FB
:1042D00012968D929C9213978D7FF601848395831D
:1042E000C3010A97DC01ED91FC911197309729F0F9
:1042F00012966D917C911397199521E0E0914833C6
:10430000F091493364807580D3018D919C91119710
:10431000848395830091483310914933F8016016E6
:10432000710609F0A3CF80859185AC014E7F40874F
:1043300051871482158282FD4EC0222331F4808180
:1043400091818017910709F046C0D80116966D90AB
:104350007C901797AD90BC901197CC24DD2476010A
:1043600029C0F5013A97848181FF21C082FD1FC0D9
:104370008680978040845184C401B301A2010E94C9
:10438000D020009741F5B201680D791DC3010E944C
:10439000C320A0E0B0E0C114D104E104F10429F08D
:1043A0008C159D05AE05BF0510F46C017D01F5016E
:1043B000A080B180A016B106A1F6D5011A96ED91A4
:1043C000FC911B97309739F01C968D919C911D970D
:1043D000B701A60119950F90DF91CF911F910F9111
:1043E000FF90EF90DF90CF90BF90AF909F908F9015
:1043F0007F906F905F904F900895E0914833F091D7
:104400004933009721F0808591858B7F03C080859B
:1044100091858460808791870895E0914833F09179
:10442000493382879387648775870895CF93DF9395
:10443000DC01FB0180839183EC0120E030E026C0A9
:10444000863271F41C9224173507FCF4F901EE0F43
:10445000FF1FEE0FFF1FE60FF71FC083D18315C0AC
:104460008D3399F4F901EE0FFF1FEE0FFF1FE60FDA
:10447000F71F80819181009741F01C922417350726
:1044800024F4C283D3832F5F3F4F119689918823F1
:10449000B9F6C901DF91CF910895AF92BF92CF9243
:1044A000DF92EF92FF920F931F93CF93DF935C0104
:1044B0006A01EB01EE24FF2400E010E00FC06881E8
:1044C00079816115710569F0C5010E94FF16009799
:1044D00011F4EA80FB800F5F1F4F24960C151D0519
:1044E00074F3C701DF91CF911F910F91FF90EF906F
:1044F000DF90CF90BF90AF9008958DE290E061E0A3
:1045000070E00E94C14689E290E062E070E00E94A3
:10451000C14689E290E00E94144784EF91E00E9436
:10452000994689E290E00E94294784E195E00E9443
:10453000994680E090E0089589E290E062E070E0C2
:104540000E94C14689E290E00E94144780E090E01A
:1045500008952DB73EB72A5030402DBF3EBFEDB76E
:10456000FEB73196ADB7BEB711968D939C93129757
:1045700085E192E28283938382E090E08483958355
:1045800016821782108611860E9480182DB73EB7BA
:10459000265F3F4F2DBF3EBF08952DB73EB7285031
:1045A00030402DBF3EBFEDB7FEB73196ADB7BEB7B9
:1045B00011968D939C9312978BE292E28283938360
:1045C00064837583468357830E9480182DB73EB756
:1045D000285F3F4F2DBF3EBF08950F931F93CF938A
:1045E000DF938C01EB010E94F016482F88A3CE01C7
:1045F000B80150E00E94E71681E090E0DF91CF9192
:104600001F910F9108950E94E7160895EF92FF926F
:104610000F931F93CF93DF930F920F92CDB7DEB717
:104620007C018B01BE016F5F7F4F40E050E00E9434
:104630003517DC01CB01F80180839183A283B3831A
:1046400001E010E020E030E089819A818E159F051D
:1046500019F400E010E09801B801C9010F900F9023
:10466000DF91CF911F910F91FF90EF9008950F93DD
:104670001F93CF93DF9300D00F92CDB7DEB78C019D
:1046800062307105CCF0FA0182819381BE016F5FC7
:104690007F4F0E940623DC01CB010097A105B105E5
:1046A00059F069817A818B819C810E94B814BC0188
:1046B000C8010E945D1910C000D00F92EDB7FEB77F
:1046C000018312838CE492E2838394830E94801896
:1046D0000F900F900F900F902496CDBFDEBFDF910B
:1046E000CF911F910F910895EF92FF920F931F9317
:1046F000CF93DF930F920F92CDB7DEB77C018B0182
:10470000BE016F5F7F4F40E050E00E943517DC0133
:10471000CB01F8018083918381E090E029813A8187
:104720002E153F0511F480E090E00F900F90DF917F
:10473000CF911F910F91FF90EF900895EF92FF920C
:104740000F931F93CF93DF930F920F92CDB7DEB7E6
:104750008C017B01BE016F5F7F4F40E050E00E9403
:104760003517AB01BC0189819A818017910741F00F
:1047700057FD06C0F7014083518381E090E002C0FD
:1047800080E090E00F900F90DF91CF911F910F91FB
:10479000FF90EF900895EF92FF920F931F93CF93A6
:1047A000DF9300D00F92CDB7DEB78C016230710578
:1047B000B4F1DA0112968D919C911397BE016F5F4F
:1047C0007F4F0E940623DC01CB010097A105B105B4
:1047D00031F169817A818B819C810E949A147C01DC
:1047E00000D000D0EDB7FEB73196ADB7BEB7119689
:1047F0000D931C93129784E792E2828393838981BD
:104800009A81848395830E948018EDB7FEB736960F
:10481000EDBFFEBFC801B7010E945D1914C000D0F2
:104820000F92ADB7BEB711960D931C93129780E807
:1048300092E213968D939C9314970E9480180F9088
:104840000F900F900F902496CDBFDEBFDF91CF91D8
:104850001F910F91FF90EF9008950F931F93CF93A7
:10486000DF930F920F92CDB7DEB78C0162307105E6
:104870009CF0FA0182819381BE016F5F7F4F0E949D
:104880007423009749F089819A810E948614BC01A3
:10489000C8010E945D1910C000D00F92EDB7FEB79D
:1048A000018312838DE992E2838394830E948018AE
:1048B0000F900F900F900F900F900F90DF91CF916E
:1048C0001F910F9108950F931F93CF93DF930F9232
:1048D000CDB7DEB78C01CE0101960E945D0ABC0106
:1048E000C8010E945D1900D000D0EDB7FEB7319627
:1048F000ADB7BEB711960D931C93129784EB92E25D
:10490000828393838981848315820E9480188DB766
:104910009EB706968DBF9EBF0F90DF91CF911F91DE
:104920000F910895CF92DF92EF92FF920F931F9312
:10493000CF93DF93CDB7DEB7A497CDBFDEBF7C01A9
:1049400025E1C22ED12CCC0EDD1ECE010196B60182
:1049500040E150E09E012B5F3F4F00E110E00E94DC
:10496000E80ABC01C7010E945D1949815A816B8127
:104970007C818DB79EB70C978DBF9EBFEDB7FEB7FC
:104980003196ADB7BEB71196ED92FC9212978AECB4
:1049900092E282839383862F90E084839583BB2762
:1049A000A72F962F852F907086839783507040870E
:1049B0005187C286D3860E9480188DB79EB70C9609
:1049C0008DBF9EBFCE0105960E94F016009719F08C
:1049D000CE01059602C082EC92E200D000D0EDB785
:1049E000FEB73196ADB7BEB71196ED92FC92129715
:1049F00029EE32E222833383848395830E948018D8
:104A00008DB79EB706968DBF9EBFA496CDBFDEBF65
:104A1000DF91CF911F910F91FF90EF90DF90CF909A
:104A20000895AF92BF92CF92DF92EF92FF920F93D1
:104A30001F93CF93DF9300D00F92CDB7DEB75C0109
:104A40008B017A01CE01019660E070E040E050E019
:104A500020E030E00E940D0CC801019785309105DF
:104A600008F070C00130110509F481C0D701129619
:104A70008D919C9113976BEF72E20E94FF16009745
:104A800009F060C00230110509F471C0F70184819A
:104A90009581BE016F5F7F4F0E940C15009709F44E
:104AA00051C00330110509F462C0D70116968D91EB
:104AB0009C91179760E070E04AE050E00E94351743
:104AC000DC01CB016C010530110521F4F7010085F3
:104AD000118502C000E010E080E0BE016F5F7F4FF3
:104AE000A60198010E941B14BC01C5010E945D191A
:104AF000CE0101960E9491160115110511F40AEFDD
:104B000012E22DB73EB72A5030402DBF3EBFEDB761
:104B1000FEB73196ADB7BEB71196AD92BC92129763
:104B200025E033E22283338384839583C682D78250
:104B3000008711870E948018EDB7FEB73A96EDBF47
:104B4000FEBF1AC000D00F92ADB7BEB71196AD929E
:104B5000BC9212978DE193E213968D939C931497D8
:104B60000E9480180F900F900F900F9005C080E961
:104B7000C82E8FE1D82EAECF2496CDBFDEBFDF91F9
:104B8000CF911F910F91FF90EF90DF90CF90BF904A
:104B9000AF9008950F931F93CF93DF93CDB7DEB7F8
:104BA0006097CDBFDEBF8C01CE010D96BE01675F61
:104BB0007F4FAE014B5F5F4F9E012F5F3F4F0E94C3
:104BC0000D0C97FD03C021E633E202C024E633E278
:104BD0004DB75EB7485050404DBF5EBFEDB7FEB712
:104BE0003196ADB7BEB711960D931C93129748E658
:104BF00053E24283538324833583868397830E94C1
:104C000080184DB75EB7485F5F4F4DBF5EBFCE01A6
:104C10000D960E94911600D000D0EDB7FEB73196E8
:104C2000ADB7BEB711960D931C93129720E733E2F0
:104C300022833383848395830E9480184DB75EB7A7
:104C40004A5F5F4F4DBF5EBFCE0109960E9491162D
:104C500000D000D0EDB7FEB73196ADB7BEB7119614
:104C60000D931C93129727E733E2228333838483C7
:104C700095830E9480184DB75EB74A5F5F4F4DBF66
:104C80005EBFCE0105960E94911600D000D0EDB710
:104C9000FEB73196ADB7BEB711960D931C93129720
:104CA00020E833E222833383848395830E94801833
:104CB0004DB75EB74A5F5F4F4DBF5EBFCE010196F5
:104CC0000E94911600D000D0EDB7FEB73196ADB777
:104CD000BEB711960D931C93129727E833E22283F7
:104CE0003383848395830E9480184DB75EB74A5FF3
:104CF0005F4F4DBF5EBF6096CDBFDEBFDF91CF91EE
:104D00001F910F9108950F931F93CF93DF9300D0BE
:104D100000D0CDB7DEB78C0162307105A4F1DA01A5
:104D200012968D919C911397BE016F5F7F4F0E94E9
:104D30007423009741F189819A81BE016D5F7F4F95
:104D40000E944A10BC01C8010E945D19CE01039661
:104D50000E94911600D000D0EDB7FEB73196ADB7E6
:104D6000BEB711960D931C93129721E933E222836B
:104D70003383848395830E948018EDB7FEB73696FF
:104D8000EDBFFEBF14C000D00F92ADB7BEB71196F5
:104D90000D931C9312978BE993E213968D939C933A
:104DA00014970E9480180F900F900F900F902696E6
:104DB000CDBFDEBFDF91CF911F910F9108952F924C
:104DC0003F924F925F926F927F928F929F92AF929B
:104DD000BF92CF92DF92EF92FF920F931F93CF93E8
:104DE000DF93CDB7DEB72897CDBFDEBF4C017B0187
:104DF0008A01643071050CF4A6C0DA0112968D9117
:104E00009C911397BE016D5F7F4F0E9474230097A2
:104E100009F499C025E0A22EB12CAC0EBD1EF801FC
:104E200084819581B5010E940C15009709F48BC00F
:104E3000D80116968D919C911797BE016F5F7F4F99
:104E40000E949E23009709F47EC0B801685F7F4FDF
:104E5000C70104970E94FF1D6C01009709F46CC004
:104E60000E94F0163C01C5010E949116EDB7FEB7F5
:104E70003A97EDBFFEBF3196ADB7BEB711968D9292
:104E80009C9212972AEB33E22283338364827582E9
:104E90008683978389819A81808791870E94801871
:104EA000EDB7FEB73A96EDBFFEBFEE24FF24250115
:104EB00096ED292E93E2392E36C05301AE18BF0865
:104EC000B6016E0D7F1D09811A818B819C81A50120
:104ED00092010E94D00F8C0197FF04C0C6010E946E
:104EE00066472CC02DB73EB7285030402DBF3EBF7F
:104EF000EDB7FEB73196ADB7BEB711968D929C92C5
:104F000012972282338284839583C501801B910B83
:104F1000868397830E948018E00EF11EEDB7FEB7DE
:104F20003896EDBFFEBFE614F7043CF2C6010E94BE
:104F3000664700E010E002C00DEF1FEFC401B801AA
:104F40000E945D1914C000D00F92ADB7BEB7119684
:104F50008D929C9212978BEE93E213968D939C9375
:104F600014970E9480180F900F900F900F90289622
:104F7000CDBFDEBFDF91CF911F910F91FF90EF90DA
:104F8000DF90CF90BF90AF909F908F907F906F9069
:104F90005F904F903F902F9008954F925F926F9245
:104FA0007F928F929F92AF92BF92CF92DF92EF92B9
:104FB000FF920F931F93CF93DF930F920F92CDB772
:104FC000DEB74C017B018A01633071050CF47CC0B3
:104FD000DA0112968D919C911397BE016F5F7F4FFE
:104FE0000E947423009709F46FC0B8016C5F7F4F73
:104FF000C70102970E94FF1D6C01009709F45DC074
:105000000E94F0165C0100D000D0EDB7FEB73196DB
:10501000ADB7BEB711968D929C9212978BE194E238
:1050200082839383A482B5820E948018EDB7FEB775
:105030003696EDBFFEBFEE24FF2436ED432E33E25D
:10504000532E32C035016E187F08B6016E0D7F1DDC
:1050500089819A81A3010E946C0F8C0197FF04C083
:10506000C6010E9466472BC08DB79EB708978DBFBB
:105070009EBFEDB7FEB73196ADB7BEB711968D9214
:105080009C9212974282538204831583C301801B32
:10509000910B868397830E948018E00EF11EEDB776
:1050A000FEB73896EDBFFEBFEA14FB045CF2C60102
:1050B0000E94664700E010E002C00DEF1FEFC40140
:1050C000B8010E945D1914C000D00F92ADB7BEB7F1
:1050D00011968D929C9212978EE294E213968D9384
:1050E0009C9314970E9480180F900F900F900F9030
:1050F0000F900F90DF91CF911F910F91FF90EF9044
:10510000DF90CF90BF90AF909F908F907F906F90E7
:105110005F904F9008950F931F93CF93DF930F925B
:105120000F92CDB7DEB78C01623071059CF0FA01A9
:1051300082819381BE016F5F7F4F0E94742300972D
:1051400049F089819A810E945E0EBC01C8010E94CB
:105150005D1910C000D00F92EDB7FEB70183128326
:1051600080E594E2838394830E9480180F900F90CF
:105170000F900F900F900F90DF91CF911F910F9193
:105180000895EF92FF920F931F93CF93DF93CDB7C4
:10519000DEB72897CDBFDEBF7C018A016430710580
:1051A00064F1FA0182819381BE016D5F7F4F0E949D
:1051B0007423009711F1F80184819581BE016B5F22
:1051C0007F4F0E940C150097C1F0F80186819781EE
:1051D000BE016F5F7F4F0E949E23009771F049814F
:1051E0005A818B819C81BE016B5F7F4F0E94D20DE3
:1051F000BC01C7010E945D1910C000D00F92EDB72D
:10520000FEB7E182F28288E694E2838394830E946F
:1052100080180F900F900F900F902896CDBFDEBF93
:10522000DF91CF911F910F91FF90EF900895CF9252
:10523000DF92EF92FF920F931F93CF93DF9300D0F3
:105240000F92CDB7DEB76C017B018A0181E090E05F
:1052500089839A836230710534F1FA0182819381E6
:10526000BE016D5F7F4F0E9474230097E1F0F2E072
:10527000EF16F10451F0F80184819581BE016F5F52
:105280007F4F0E947423009771F069817A818B812E
:105290009C814FE659E296010E94970DBC01C60120
:1052A0000E945D1910C000D00F92EDB7FEB7C18209
:1052B000D2828EE894E2838394830E9480180F90B8
:1052C0000F900F900F902496CDBFDEBFDF91CF914E
:1052D0001F910F91FF90EF90DF90CF9008950F9363
:1052E0001F93CF93DF938C01EB0100D000D0EDB77B
:1052F000FEB73196ADB7BEB711968D939C931297BA
:1053000081EB94E282839383648375830E94801887
:105310008DB79EB706968DBF9EBFCE010E94140E1C
:10532000EC01181619065CF46DEC72E2A8010E94FB
:10533000320DCE0168EA79E2A8010E944B0DC80146
:10534000BE010E945D19DF91CF911F910F910895C9
:10535000AF92BF92CF92DF92EF92FF920F931F9383
:10536000CF93DF93CDB7DEB7C054D040CDBFDEBF03
:105370006C015B018A014115510519F08AEF92E237
:1053800002C085ED94E22DB73EB72A5030402DBFC4
:105390003EBFEDB7FEB73196ADB7BEB71196CD9211
:1053A000DC92129727EE34E222833383A482B58203
:1053B00006831783808791870E9480182DB73EB798
:1053C000265F3F4F2DBF3EBF15C0C501BE016F5FB9
:1053D0007F4FA7010E94B60E9C0118161906ACF764
:1053E000081B190BC60165E075E2AE014F5F5F4F08
:1053F0000E94C119101611064CF40134110518F061
:1054000080E490E001C0C8017C01DFCFC05CDF4FC9
:10541000CDBFDEBFDF91CF911F910F91FF90EF9035
:10542000DF90CF90BF90AF900895EF92FF920F93CF
:105430001F93CF93DF93CDB7DEB72897CDBFDEBFE5
:105440007C018A016430710564F1FA0182819381E3
:10545000BE016D5F7F4F0E947423009711F1F80128
:1054600084819581BE016B5F7F4F0E940C15009770
:10547000C1F0F80186819781BE016F5F7F4F0E9466
:105480009E23009771F049815A818B819C81BE01D6
:105490006B5F7F4F0E94640DBC01C7010E945D19C4
:1054A00010C000D00F92EDB7FEB7E182F28288E023
:1054B00095E2838394830E9480180F900F900F9041
:1054C0000F902896CDBFDEBFDF91CF911F910F9136
:1054D000FF90EF900895AF92BF92CF92DF92EF923C
:1054E000FF920F931F93CF93DF930F920F92CDB73D
:1054F000DEB76C015B018A0119821A826230710584
:105500000CF449C0FA01828193816BE275E20E943A
:10551000FF160097B1F0F8018281938162E375E292
:105520000E94FF16009781F0F8018281938168E361
:1055300075E20E94FF16009771F552E0E52EF12CFE
:1055400006C0EE24FF2403C041E0E42EF12CF2E07B
:10555000AF16B10451F0F80184819581BE016F5FEF
:105560007F4F0E9474230097B1F069817A81C7014F
:105570000E94DB0C8C016DEC72E2A6010E94320DE0
:10558000C80168EA79E2A6010E944B0DC601B80184
:105590000E945D1910C000D00F92EDB7FEB7C18216
:1055A000D2828CE395E2838394830E9480180F90CB
:1055B0000F900F900F900F900F90DF91CF911F9150
:1055C0000F91FF90EF90DF90CF90BF90AF90089534
:1055D0000F931F93CF93DF930F920F92CDB7DEB748
:1055E0008C01623071059CF0FA0182819381BE01C9
:1055F0006F5F7F4F0E947423009749F089819A81E1
:105600000E944E0CBC01C8010E945D1910C000D060
:105610000F92EDB7FEB7018312838AE695E283838A
:1056200094830E9480180F900F900F900F900F900E
:105630000F90DF91CF911F910F9108950F931F93BA
:10564000CF93DF930F920F92CDB7DEB78C01CE01CF
:1056500001960E94320C97FD03C021E633E202C09E
:1056600024E633E24DB75EB74A5050404DBF5EBFAF
:10567000EDB7FEB73196ADB7BEB711960D931C933B
:10568000129743E855E2428353832483358386830C
:10569000978389819A81808791870E9480184DB76E
:1056A0005EB7465F5F4F4DBF5EBF0F900F90DF91BB
:1056B000CF911F910F9108950F931F93CF93DF9375
:1056C0000F920F92CDB7DEB78C01623071059CF05E
:1056D000FA0182819381BE016F5F7F4F0E94742324
:1056E000009749F089819A810E94220CBC01C8016F
:1056F0000E945D1910C000D00F92EDB7FEB7018374
:10570000128388E995E2838394830E9480180F9026
:105710000F900F900F900F900F90DF91CF911F91EE
:105720000F910895CF92DF92EF92FF920F931F9304
:10573000CF93DF93CDB7DEB76097CDBFDEBF6C01EF
:105740007B018A018091F9319091FA31A091FB316E
:10575000B091FC3189879A87AB87BC878D839E8304
:10576000AF83B88789839A83AB83BC83623071052A
:105770000CF446C0FA0182819381BE01635F7F4FC2
:105780000E940C150097E1F1F2E0EF16F10431F1FF
:10579000F80184819581BE01675F7F4F0E940C15DF
:1057A000009771F1F3E0EF16F104C1F0F801868182
:1057B0009781BE016B5F7F4F0E940C15009701F12E
:1057C000F4E0EF16F10451F0F80180859185BE01F7
:1057D0006F5F7F4F0E940C15009791F0CE010D96E0
:1057E000BE01675F7F4FAE014B5F5F4F9E012F5F32
:1057F0003F4F0E94040CBC01C6010E945D1910C0FD
:1058000000D00F92EDB7FEB7C182D28280EB95E255
:10581000838394830E9480180F900F900F900F90B5
:105820006096CDBFDEBFDF91CF911F910F91FF90AA
:10583000EF90DF90CF900895EF92FF920F931F9318
:10584000CF93DF93CDB7DEB7CF54D040CDBFDEBF0F
:105850007C01CE0182960E94940C8C0197FD03C0BE
:1058600081E693E202C084E693E22DB73EB728506A
:1058700030402DBF3EBFEDB7FEB73196ADB7BEB7D6
:105880001196ED92FC9212972FED35E2228333832D
:1058900084839583068317830E948018EDB7FEB733
:1058A0003896EDBFFEBF0115110579F000D00F92BB
:1058B000ADB7BEB71196ED92FC92129785EE95E2C8
:1058C00013968D939C931497C7C023964FAD23973F
:1058D000CE010196BE016E5D7F4F50E00E94E7163B
:1058E00023968FAD2397E1E0F0E0EC0FFD1FE80F6A
:1058F000F11D1082882319F0CE01019602C08BEDB4
:1059000095E2EDB7FEB77297EDBFFEBF3196ADB72A
:10591000BEB71196ED92FC92129728EE35E22283E3
:1059200033838483958327968FAD27978683178249
:1059300028968FAD28978087118629968FAD299755
:10594000828713862A968FAD2A97848715862B9691
:105950008FAD2B97868717862C968FAD2C97808BD3
:10596000118A0E9480182E968EAD9FAD2E97EDB7AE
:10597000FEB77296EDBFFEBFFFEF80389F07C9F0FC
:1059800000D000D0EDB7FEB73196ADB7BEB71196D7
:10599000ED92FC9212972CE036E2228333838483CB
:1059A00095830E948018EDB7FEB73696EDBFFEBF17
:1059B00014C000D00F92ADB7BEB71196ED92FC9215
:1059C000129785E196E213968D939C9314970E940B
:1059D00080180F900F900F900F9060968EAD9FAD36
:1059E0006097BFEF80389B07C9F000D000D0EDB7BB
:1059F000FEB73196ADB7BEB71196ED92FC921297F5
:105A00002FE136E222833383848395830E948018BA
:105A1000EDB7FEB73696EDBFFEBF14C000D00F92B3
:105A2000ADB7BEB71196ED92FC92129786E296E260
:105A300013968D939C9314970E9480180F900F904B
:105A40000F900F9000D00F92EDB7FEB7E182F28277
:105A50008EE296E2838394830E9480180F900F90C9
:105A60000F900F90C15BDF4FCDBFDEBFDF91CF91B5
:105A70001F910F91FF90EF9008950F931F93CF9375
:105A8000DF9300D000D0CDB7DEB78C01CE010196F8
:105A90000E94670C97FD03C021E633E202C024E6B2
:105AA00033E24DB75EB7445150404DBF5EBFEDB7D6
:105AB000FEB73196ADB7BEB711960D931C931297F2
:105AC00042E356E24283538324833583868397835C
:105AD0008981808711868A81828713868B8184875A
:105AE00015868C81868717868D81808B118A8E81A1
:105AF000828B138A0E9480184DB75EB74C5E5F4F51
:105B00004DBF5EBF2696CDBFDEBFDF91CF911F9107
:105B10000F9108950F931F93CF93DF930F920F92DE
:105B2000CDB7DEB78C0162307105B4F0FA01828125
:105B30009381BE016F5F7F4F0E947423009761F0D5
:105B4000898160E070E040E050E00E94AC13BC014D
:105B5000C8010E945D1910C000D00F92EDB7FEB7CA
:105B6000018312838AE596E2838394830E948018DE
:105B70000F900F900F900F900F900F90DF91CF919B
:105B80001F910F910895CF92DF92EF92FF920F93A2
:105B90001F93CF93DF9300D000D0CDB7DEB76C0159
:105BA0007B018A0164307105ACF1FA018281938135
:105BB000BE016B5F7F4F0E947423009759F1F8017B
:105BC00084819581BE016D5F7F4F0E947423009791
:105BD00009F1F80186819781BE016F5F7F4F0E94B6
:105BE00074230097B9F0F4E0EF16F10421F0F80106
:105BF0002085318502C020E030E06B817C814981C5
:105C00005A818D819E810E94BC13BC01C6010E94F5
:105C10005D191AC000D00F92EDB7FEB7C182D282D3
:105C200089E796E2838394830E948018EDB7FEB7DC
:105C3000C182D28282EA96E2838394830E94801892
:105C40000F900F900F900F902696CDBFDEBFDF9183
:105C5000CF911F910F91FF90EF90DF90CF9008951B
:105C6000AF92BF92CF92DF92EF920F931F93CF9399
:105C7000DF93CDB7DEB76097CDBFDEBF5C018A0191
:105C80006630710509F052C0FA0182819381BE012C
:105C90006D5F7F4F0E947423009709F447C0F8019D
:105CA00084819581BE01635F7F4F0E940623DC01E2
:105CB000CB010097A105B105C9F1F8018681978153
:105CC000BE01675F7F4F0E940623DC01CB01009776
:105CD000A105B10559F1F80180859185BE016F5F7D
:105CE0007F4F0E947423009709F1F8018285938504
:105CF000BE016B5F7F4F0E940623DC01CB01009742
:105D0000A105B10599F04D855E856F857889098576
:105D10001A852B853C85CD80DE808B81E9800E94B1
:105D2000D313BC01C5010E945D191AC000D00F92A7
:105D3000EDB7FEB7A182B2828AEC96E283839483A8
:105D40000E948018EDB7FEB7A182B2828EEF96E274
:105D5000838394830E9480180F900F900F900F9070
:105D60006096CDBFDEBFDF91CF911F910F91EF9075
:105D7000DF90CF90BF90AF9008950F931F93CF9374
:105D8000DF930F920F92CDB7DEB78C0162307105B1
:105D90009CF0FA0182819381BE016F5F7F4F0E9468
:105DA0007423009749F089819A810E94BF13BC0136
:105DB000C8010E945D1910C000D00F92EDB7FEB768
:105DC000018312838AE397E2838394830E9480187D
:105DD0000F900F900F900F900F900F90DF91CF9139
:105DE0001F910F9108950F931F93CF93DF930F92FD
:105DF000CDB7DEB78C01CE0101960E948F139C01B6
:105E0000E981E33040F4F0E0EE0FFF1FE95FFC4C66
:105E10008081918102C080E090E037FF05C044E6B8
:105E200053E28BED95E202C041E653E26DB77EB7D7
:105E30006A5070406DBF7EBFEDB7FEB73196ADB70B
:105E4000BEB711960D931C93129760E577E26283BB
:105E500073834483558326833783808791870E9489
:105E600080186DB77EB7665F7F4F6DBF7EBF0F90A6
:105E7000DF91CF911F910F9108950F931F93CF93AF
:105E8000DF930F920F92CDB7DEB78C0162307105B0
:105E90009CF0FA0182819381BE016F5F7F4F0E9467
:105EA0007423009749F089819A810E943C13BC01B8
:105EB000C8010E945D1910C000D00F92EDB7FEB767
:105EC000018312838DE597E2838394830E94801877
:105ED0000F900F900F900F900F900F90DF91CF9138
:105EE0001F910F910895CF93DF93EC010E947218D8
:105EF000BC0183E093E20E944C13BC01CE010E94DE
:105F00005D19DF91CF910895CF93DF93EC010E944B
:105F100072180E946713BC01CE010E945D19DF91C7
:105F2000CF910895CF93DF93EC010E94F60BBC0153
:105F3000CE010E945D19DF91CF910895CF92DF923B
:105F4000EF92FF920F931F93CF93DF93CDB7DEB7FE
:105F5000A197CDBFDEBF6C018B017A01CE01019606
:105F600060E070E041E250E00E94EA160430110562
:105F700094F1F70182819381BE016F5F7F4F0E9490
:105F8000ED22009709F45AC0F70106811781C80174
:105F900064E777E20E94FF16009791F0C80169E775
:105FA00077E20E94FF16009771F0C8016DE777E273
:105FB0000E94FF16009709F041C041E050E005C083
:105FC00043E050E002C042E050E0F7016481758197
:105FD000CE0101962CC00330110581F4F7018281B6
:105FE0009381BE016F5F7F4F0E94ED22009731F1D8
:105FF000F70164817581CE01019617C00230110549
:1060000069F4F70182819381BE016F5F7F4F0E9427
:10601000ED22009799F0CE01019605C001301105DF
:1060200069F480E090E060E070E040E050E00E94C1
:106030009C0BBC01C6010E945D1910C000D00F92DC
:10604000EDB7FEB7C182D28281E897E28383948361
:106050000E9480180F900F900F900F90A196CDBFC7
:10606000DEBFDF91CF911F910F91FF90EF90DF90F6
:10607000CF9008958F929F92AF92BF92CF92DF926E
:10608000EF92FF920F931F93CF93DF9300D000D036
:10609000CDB7DEB74C018A011B821C821D821E8295
:1060A00019821A8263307105E4F0DA0112968D913B
:1060B0009C911397BE016D5F7F4F0E940623DC0108
:1060C000CB010097A105B10509F446C0F801848110
:1060D0009581BE016F5F7F4F0E9474230097A1F4EA
:1060E0003BC062307105C1F5DA0112968D919C9129
:1060F0001397BE016D5F7F4F0E940623DC01CB0129
:106100000097A105B10541F16B817C818D819E8154
:1061100049810E94BE0A5C010097C9F48AEF90E0B1
:106120000E9499464B815C816D817E81C980DA80B5
:1061300080914E3390914F3328E030E000E010E042
:10614000E1E0EE2EF12C0E94204597FD16C0C4011F
:10615000B5010E945D1929C000D00F92EDB7FEB7BE
:10616000818292828DEA97E2838394830E948018D1
:106170000F900F900F900F9018C000D000D0EDB787
:10618000FEB73196ADB7BEB711968D929C9212971D
:1061900027ED37E222833383848395830E9480181E
:1061A000EDB7FEB73696EDBFFEBF2696CDBFDEBF7C
:1061B000DF91CF911F910F91FF90EF90DF90CF90E3
:1061C000BF90AF909F908F9008950F931F93CF93A0
:1061D000DF93CDB7DEB7A197CDBFDEBF8C016230B4
:1061E00071056CF0FA0182819381BE016F5F7F4F70
:1061F0000E94ED22009731F1CE01019602C080E0AD
:1062000090E06AE371E3A8010E945E0BBC01C80143
:106210000E945D19C8010E947618009719F500D0F8
:106220000F92EDB7FEB70183128380E098E283837B
:1062300094830E948018EDB7FEB70183128388E330
:1062400098E208C000D00F92EDB7FEB70183128329
:1062500080E898E2838394830E9480180F900F90C7
:106260000F900F90A196CDBFDEBFDF91CF911F9110
:106270000F910895CF92DF92EF92FF920F931F93A9
:10628000CF93DF93CDB7DEB7A197CDBFDEBF7C0143
:106290008B016115710509F433C10E9476180097CE
:1062A00009F02EC12DB73EB7205130402DBF3EBF63
:1062B000EDB7FEB73196ADB7BEB71196ED92FC9231
:1062C000129780EA98E282839383D80194968C9106
:1062D00094978483158295968C91959786831782DF
:1062E00096968C9196978087118697968C91979722
:1062F0008287138698968C919897848715869996AD
:106300008C91868717860E948018EDB7FEB770962D
:10631000EDBFFEBFD80193968C919397882319F413
:1063200084E998E202C08AE998E2EDB7FEB73A97AD
:10633000EDBFFEBF3196ADB7BEB71196ED92FC92A0
:10634000129720EC38E22283338384839583D8012B
:1063500092968C919297868317829A968D919C91B2
:106360009B97808791870E948018F80184A595A546
:106370002DB73EB7265F3F4F2DBF3EBF3FEF803862
:106380009307C9F000D000D0EDB7FEB73196ADB796
:10639000BEB71196ED92FC92129720ED38E222835F
:1063A0003383848395830E948018EDB7FEB73696B9
:1063B000EDBFFEBF14C000D00F92ADB7BEB71196AF
:1063C000ED92FC92129788ED98E213968D939C9330
:1063D00014970E9480180F900F900F900F90F80163
:1063E00081A1823021F1833030F4882361F0813043
:1063F00009F050C013C0843071F1843018F1853039
:1064000009F048C037C000D00F92ADB7BEB71196A3
:10641000ED92FC9212978EED98E227C000D00F9279
:10642000EDB7FEB7E182F28289EE98E22BC000D090
:106430000F92ADB7BEB71196ED92FC92129784EF12
:1064400098E213C000D00F92EDB7FEB7E182F2825E
:106450008FEF98E217C000D00F92ADB7BEB711967C
:10646000ED92FC9212978AE099E213968D939C9399
:1064700014970AC000D00F92EDB7FEB7E182F28206
:1064800085E199E2838394830E9480180F900F9096
:106490000F900F906E010894C11CD11CC60160E0E2
:1064A00070E041E250E00E94EA16D80190964C91CB
:1064B000C601B80150E00E94E71600D000D0EDB749
:1064C000FEB73196ADB7BEB71196ED92FC9212971A
:1064D00080E299E282839383C482D5820E948018ED
:1064E0000F900F90EDB7FEB7E182F28285EE95E254
:1064F000838394830E9480180F900F900F900F90C9
:10650000A196CDBFDEBFDF91CF911F910F91FF907C
:10651000EF90DF90CF900895CF93DF93EC01CB0104
:106520000097A9F400D00F92ADB7BEB71196CD93E6
:10653000DC93129783E299E213968D939C931497C0
:106540000E9480180F900F900F900F901AC00E9419
:10655000911600D000D0EDB7FEB73196ADB7BEB7FB
:106560001196CD93DC9312972FE339E22283338384
:10657000848395830E948018EDB7FEB73696EDBFF1
:10658000FEBFDF91CF910895CF93DF93EC0162308E
:1065900071056CF0FA01828193816CE872E3AE01BF
:1065A0000E947410BC01CE010E945D1910C000D081
:1065B0000F92EDB7FEB78183928381E599E28383E1
:1065C00094830E9480180F900F900F900F90DF918E
:1065D000CF9108950F931F93CF93DF938C01EA011E
:1065E0006230710524F18A819B8163E779E20E9420
:1065F000FF16009791F08A819B8167E779E20E94FC
:10660000FF16009761F08A819B816AE779E20E9418
:10661000FF16009761F482E003C080E001C081E0D2
:106620000E947F13BC01C8010E945D1910C000D0F8
:106630000F92EDB7FEB70183128380E899E283835E
:1066400094830E9480180F900F900F900F90DF910D
:10665000CF911F910F910895CF93DF93EC01888123
:106660009981009721F00E945E0E18821982DF91B5
:10667000CF9108950F931F93CF93DF938C01FC016B
:1066800082819381009721F0C80102960E942C33E9
:10669000F801808191810E94140EEC0197FD0EC0DB
:1066A00069ED73E3A8010E94320DCE0163E673E346
:1066B000A8010E944B0DF801C283D383DF91CF91D3
:1066C0001F910F910895AF92BF92CF92DF92EF92F8
:1066D000FF920F931F93CF93DF938C015B01EA012D
:1066E000209709F457C086E0C82ED12CC00ED11EC9
:1066F000CB01B60140E850E00E94B60E7C01AE012D
:10670000481B590BC50160E070E00E94B60EF7FC13
:1067100045C0F80182819381009709F43FC0EE0DD6
:10672000FF1D1582C60167E07EE20E9441170097B7
:10673000A9F1C6016AE07EE244E050E00E94FC1646
:10674000009741F59801265F3F4FC901F90140814B
:106750002F5F3F4F4C30C9F34A30B9F34D30A9F3A6
:10676000493099F34B3089F3403279F3DF012191BD
:106770002C3051F02A3041F02D3031F0293021F009
:106780002B3011F0203291F71C92F8016281738155
:106790000E946041C80102960E942C33DF91CF9184
:1067A0001F910F91FF90EF90DF90CF90BF90AF902F
:1067B0000895CF93DF9300D00F92CDB7DEB79C0141
:1067C000CB014115510531F0BE016F5F7F4F0E9433
:1067D0004A1004C0C90102960E942C332496CDBFF2
:1067E000DEBFDF91CF9108950F931F93CF93DF9377
:1067F0008C0186E890E00E944E47EC01009739F149
:1068000080E090E060E070E00E94DB0C8883998378
:1068100097FD12C069EF71E3A8010E94640D009713
:1068200059F48881998161E070E04AE353E39E0165
:106830000E94970D009759F088819981009711F077
:106840000E945E0ECE010E946647C0E0D0E0CE01FD
:10685000DF91CF911F910F910895CF93DF93EC01BA
:1068600002960E942C3388819981009711F00E9432
:106870005E0ECE010E946647DF91CF910895EF92A0
:10688000FF920F931F93CF93DF93EC01CB017A011B
:1068900089010E94911600D000D0EDB7FEB7319665
:1068A000ADB7BEB71196CD93DC9312972FE03EE2C1
:1068B00022833383848395830E9480180F920F92E2
:1068C000EDB7FEB73196ADB7BEB71196CD93DC9359
:1068D00012978CE29EE282839383E482F5820683A0
:1068E00017830E9480188DB79EB708968DBF9EBFF4
:1068F000DF91CF911F910F91FF90EF900895CF936B
:10690000DF93EC01888D998D1816190614F40E94F6
:106910005E0E8A8D9B8D009711F00E949C208C81C9
:106920009D810E946647CE010E946647DF91CF910C
:106930000895CF92DF92EF92FF920F931F93CF9320
:10694000DF93EB010C811D81888999892A893B8914
:106950008217930779F4EA85FB85309739F04C89E3
:106960005D892E893F898C859D851995CE010E9470
:106970007F347EC0EE80FF8088E090E0E80EF91E54
:1069800088E0F80180831182128213828E859F85B0
:106990000E94D614F80184839583888999890E947E
:1069A000D614F80186839783970140E050E0BA013E
:1069B0000FC0D080CC24818190E08C299D29329613
:1069C000A0E0B0E0480F591F6A1F7B1F22503040E3
:1069D0002230310570F7C70196958795FC01EE0FBF
:1069E000FF1FE00FF11F880F991FE816F90641F00D
:1069F000908180E0A0E0B0E0480F591F6A1F7B1F24
:106A0000CB01AA27BB2760707070480F591F6A1FFF
:106A10007B1F60FF09C0CB01AA27BB276070707085
:106A2000480F591F6A1F7B1FCA010E94D614809508
:106A30009095F80182839383888D998DB801A70181
:106A40009E0100E010E00E94D00F8E159F0529F4F2
:106A50008C899D8901968C8B9D8B8A8D9B8D68EE90
:106A600073E00E949F20888999890196888B998B71
:106A7000DF91CF911F910F91FF90EF90DF90CF901A
:106A80000895AF92BF92CF92DF92EF92FF920F9351
:106A90001F93CF93DF93EC016B018A01CA010E941F
:106AA0004B477C010097A1F1C601B701A8010E94E4
:106AB000B60E6C018017910759F58CE1C816D10408
:106AC0003CF1F701808D918D0E94DA142E853F856F
:106AD00082179307E9F48E899F8901968E8B9F8B8D
:106AE000A884B984A114B10499F00C84DD85C02D6B
:106AF000F701828D938D0E94DA149C01A701445FF7
:106B00005F4FF7010489CE01B60110E0F501199538
:106B1000C7010E946647DF91CF911F910F91FF90AF
:106B2000EF90DF90CF90BF90AF900895CF92DF921B
:106B3000EF92FF920F931F93CF93DF93EC016B01C2
:106B4000CA01790101151105A1F40E9491162DB712
:106B50003EB72A5030402DBF3EBFEDB7FEB731964D
:106B6000ADB7BEB71196CD93DC93129722E53EE206
:106B700013C003301105F9F40E949116ADB7BEB7EA
:106B80001A97ADBFBEBFEDB7FEB731961196CD9344
:106B9000DC93129722E73EE222833383C482D582BC
:106BA00086839783E086F1860E9480182DB73EB7D2
:106BB000265F3F4F20C00E949116ADB7BEB71C970D
:106BC000ADBFBEBFEDB7FEB731961196CD93DC9346
:106BD00012972FEA3EE222833383C482D5828683D2
:106BE0009783E086F186028713870E9480182DB76D
:106BF0003EB7245F3F4F2DBF3EBFDF91CF911F9126
:106C00000F91FF90EF90DF90CF9008954F925F9299
:106C10006F927F928F929F92AF92BF92CF92DF92AC
:106C2000EF92FF920F931F93CF93DF930F920F92E8
:106C3000CDB7DEB75C013B01490168018CE190E012
:106C400049835A830E944E472C0149815A810097FB
:106C500009F442C08A01C80108960E944E47F20119
:106C6000848395830097A9F182E090E061E070E071
:106C70000E94DB0CF201808F918F181619064CF5DB
:106C800061E475E3A2010E944B0DF50180819181C1
:106C9000A281B381F20180839183A283B383628A4C
:106CA000738A068317831686178680869186C28626
:106CB000D386E486F58680E090E060E070E049E904
:106CC00054E392010E947820F201828F938F009703
:106CD00031F4C2010E947F348DEF9FEF02C080E04B
:106CE00090E00F900F90DF91CF911F910F91FF9047
:106CF000EF90DF90CF90BF90AF909F908F907F905C
:106D00006F905F904F9008954F925F926F927F9235
:106D10008F929F92AF92BF92CF92DF92EF92FF92AB
:106D20000F931F93CF93DF9300D00F92CDB7DEB7B1
:106D30002C016B015A018091F9319091FA31A091A7
:106D4000FB31B091FC3189839A83AB83BC83E1E052
:106D5000EE2EF12CF0E26F2E712C13E0812E912C8F
:106D600055C08701000F111F0A0D1B1DD8018D9101
:106D70009C916EED7EE20E94FF160097C1F408948C
:106D8000E11CF11CEC14FD040CF08DC0F701EE0FBA
:106D9000FF1FEA0DFB1D8081918160E070E04AE0F9
:106DA00050E00E943517DC01CB014C012CC0F801EA
:106DB0008081918161EE7EE20E94FF160097C1F40E
:106DC0000894E11CF11CEC14FD040CF06CC0F701FC
:106DD000EE0FFF1FEA0DFB1D8081918160E070E0E6
:106DE0004AE050E00E943517DC01CB013C010BC0AA
:106DF000D8018D919C91BE016F5F7F4F0E940C1551
:106E0000009709F450C00894E11CF11CEC14FD0437
:106E10000CF4A7CF89819A81AB81BC814091F93173
:106E20005091FA316091FB317091FC3184179507D4
:106E3000A607B707C1F1CE010196B401A30126E967
:106E400035E30FE314E372010E9406368C0197FDCF
:106E500005C087EDE82E8EE2F82E04C0BAEDEB2EC9
:106E6000BEE2FB2EC8010E948E1FEDB7FEB73A9717
:106E7000EDBFFEBF3196ADB7BEB711964D925C9295
:106E8000129724EE3EE222833383E482F582068366
:106E90001783808791870E948018EDB7FEB73A96D6
:106EA000EDBFFEBF14C000D00F92ADB7BEB71196B4
:106EB0004D925C92129781EF9EE213968D939C9374
:106EC00014970E9480180F900F900F900F902496A7
:106ED000CDBFDEBFDF91CF911F910F91FF90EF905B
:106EE000DF90CF90BF90AF909F908F907F906F90EA
:106EF0005F904F9008958F929F92AF92BF92CF92E2
:106F0000DF92EF92FF920F931F93CF93DF93EC01E9
:106F1000D62EC72E88899989009779F02C813D81DA
:106F20008E819F81289FA001299F500D389F500D71
:106F300011244A01AA24BB2404C08A889B88AC88F7
:106F4000BD886C857D85888599850E94C320EA8DE2
:106F5000FB8D309751F07C0100E010E08C8D9D8D11
:106F60006D2D7C2DA501940119958A819B810E942C
:106F70006647888199810E945E0E88899989009769
:106F800021F48E899F890E945E0ECE010E94664781
:106F90008D2D9C2DDF91CF911F910F91FF90EF9040
:106FA000DF90CF90BF90AF909F908F9008956F9299
:106FB0007F928F929F92AF92BF92CF92DF92EF9289
:106FC000FF920F931F93CF93DF93EC013B01490195
:106FD0005A016701780100D00F92ADB7BEB7119684
:106FE0008D939C93129782E29FE213968D939C93CC
:106FF00014970E9480180F900F900F900F906114BB
:107000007104C1F0C3010E948E1FEDB7FEB738971F
:10701000EDBFFEBF3196ADB7BEB71196CD93DC93F1
:10702000129725E23FE2228333836482758286834E
:1070300097834AC02DB73EB7C114D104E104F104CF
:1070400071F1205130402DBF3EBF0DB71EB70F5F0D
:107050001F4FADB7BEB71196CD93DC93129788E35F
:107060009FE2F8018283938384829582A682B7820D
:10707000C086D186E286F386C501B401A7019601D8
:107080000E941A51D8011C962D933D934D935C9309
:107090001F970E948018EDB7FEB770961AC028504F
:1070A00030402DBF3EBFEDB7FEB73196ADB7BEB78E
:1070B0001196CD93DC9312978BE69FE282839383A4
:1070C00084829582A682B7820E948018EDB7FEB7AF
:1070D0003896EDBFFEBFDF91CF911F910F91FF90CA
:1070E000EF90DF90CF90BF90AF909F908F907F9068
:1070F0006F9008950F931F93CF93DF938C01EB0153
:1071000000D00F92EDB7FEB78183928382E99FE2B0
:10711000838394830E9480180F900F900F900F909C
:107120001C161D06BCF4CE0160E570E00E940751FC
:10713000009781F400D00F92EDB7FEB70183128360
:1071400082E29FE2838394830E9480180F900F90C5
:107150000F900F90DF91CF911F910F910895CF93D2
:10716000DF93EC01CB010E94140EBC018E8B9F8B30
:1071700097FF04C0CE010E947B3714C06CE179E315
:10718000AE010E94320D8E899F8965ED78E3AE01D4
:107190000E944B0D0E94AF20A0E0B0E08887998745
:1071A000AA87BB87DF91CF910895CF93DF93EC013E
:1071B0009B01888999890097E1F54115510561F492
:1071C0000E94AF20A0E0B0E08C879D87AE87BF878C
:1071D000CE0160E070E00BC06A817B814C815D81F3
:1071E000C9010E94B60EBC0197FF04C0CE010E94E7
:1071F0007B371FC02E813F812F5F3F4F2E833F8300
:10720000CB01AA2797FDA095BA2F4A895B896C8983
:107210007D89480F591F6A1F7B1F4A8B5B8B6C8BC4
:107220007D8BE88DF98D309721F08C8D9D8DB90186
:107230001995DF91CF910895EF92FF920F931F93CD
:10724000CF93DF93EC014115510519F46CEF7FEFFB
:107250003CC00E94AF20A0E0B0E088879987AA8751
:10726000BB87EE24FF2421C06A817B81600F711FE0
:10727000401B510B888199810E946C0FBC0197FDC6
:107280000BC0080F191F02C000E010E04C815D81A7
:107290000417150748F322C0CE0117C08C8D9D8DB1
:1072A000B70119950894E11CF11C8E819F81E816A5
:1072B000F90650F30E94AF20A0E0B0E08C879D87D4
:1072C000AE87BF87CE0160E070E00E947B37DF9120
:1072D000CF911F910F91FF90EF900895E88DF98D58
:1072E0003097E1F6DFCF4F925F926F927F928F924D
:1072F0009F92AF92BF92CF92DF92EF92FF920F9345
:107300001F93CF93DF932C013B01EA015901480100
:10731000209709F456C02115310509F452C06115B2
:10732000710509F44EC08EE190E00E944E478C0139
:10733000009709F449C0FC01C683D783A482B582B3
:10734000808E918EE28EF38EC48ED58E81E090E099
:10735000808B918BC5010E944B47F80182839383F8
:10736000009721F4C8016DEF7FEF0DC080E090E041
:1073700060E070E00E94DB0CBC01F8018083918327
:1073800097FF04C0C8010E947B3720C0B201A3014F
:107390000E94D20DBC0197FDF5CFF801808191814B
:1073A0006CE179E3A8010E94320DF801808191819E
:1073B00065ED78E3A8010E944B0DF8018081918171
:1073C00005C08EEF9FEF02C08DEF9FEFDF91CF9151
:1073D0001F910F91FF90EF90DF90CF90BF90AF90F3
:1073E0009F908F907F906F905F904F9008958F92B5
:1073F0009F92AF92BF92CF92DF92EF92FF920F9344
:107400001F93CF93DF934C017B015A0169018EE1F9
:1074100090E00E944E47EC01009719F480E090E064
:1074200010C0EC82FD82A88EB98ECA8EDB8E0C8FC6
:107430001D8FC7010E944B478A839B83009731F4BD
:10744000CE016DEF7FEF0E947B3723C080E090E09C
:1074500060E070E00E94DB0CBC018883998397FD9B
:1074600014C069EF71E3A4010E94640DBC0197FD93
:107470000CC08881998161E070E04FEA58E39E0179
:107480000E94970DBC0197FF02C0CE01DCCF88811E
:107490009981DF91CF911F910F91FF90EF90DF9035
:1074A000CF90BF90AF909F908F9008952F923F9272
:1074B0004F925F926F927F928F929F92AF92BF9204
:1074C000CF92DF92EF92FF920F931F93CF93DF93B0
:1074D00000D000D0CDB7DEB75C016B014A018091CE
:1074E000F9319091FA31A091FB31B091FC3189834F
:1074F0009A83AB83BC8322243324412C24E0522E74
:1075000020E034E02D833E83E8E86E2EE3E17E2E1A
:10751000F1E0EF2EF12C8FC08701000F111F080D35
:10752000191DD8018D919C9164E97FE20E94FF169C
:107530000097C1F40894E11CF11CEC14FD040CF05C
:1075400019C1F701EE0FFF1FE80DF91D8081918130
:1075500060E070E04AE050E00E943517DC01CB01AA
:107560003C0166C0F8018081918167E97FE20E9459
:10757000FF160097C9F40894E11CF11CEC14FD04FB
:107580000CF0F8C0F701EE0FFF1FE80DF91D808128
:10759000918160E070E04AE050E00E943517DC0124
:1075A000CB018D839E8344C0D8018D919C916AE963
:1075B0007FE20E94FF160097C1F40894E11CF11CC1
:1075C000EC14FD040CF0D6C0F701EE0FFF1FE80D20
:1075D000F91D8081918160E070E04AE050E00E94F6
:1075E0003517DC01CB012C0123C0F801808191818A
:1075F0006DE97FE20E94FF160097A1F0D8018D91FE
:107600009C9160EA7FE20E94FF16009779F0F801F2
:1076100080819181BE016F5F7F4F0E940C150097A2
:1076200039F4A8C0F1E02F2E312C02C022243324DB
:107630000894E11CF11CEC14FD040CF46DCF211432
:10764000310411F189819A81AB81BC814091F9317A
:107650005091FA316091FB317091FC31841795079C
:10766000A607B70709F486C0CE010196B3014D8184
:107670005E8192010AE718E3E7EDEE2EE7E3FE2EC6
:1076800065010E94733909C0C301B2014AE758E39A
:1076900027ED37E385010E94F7398C0197FF1EC063
:1076A0000E948E1F2DB73EB72A5030402DBF3EBFDF
:1076B000EDB7FEB73196ADB7BEB71196AD92BC929D
:1076C000129723EA3FE22283338320EB3FE22483B5
:1076D0003583068317838087918744C02114310442
:1076E00059F1CE0101960E9491162DB73EB72E504A
:1076F00030402DBF3EBFEDB7FEB73196ADB7BEB738
:107700001196AD92BC92129724EB3FE22283338311
:1077100084839583668277822D813E81208731879D
:1077200042865386048715870E9480188DB79EB7BE
:107730000E968DBF9EBF32C0ADB7BEB71A97ADBF14
:10774000BEBFEDB7FEB731961196AD92BC921297BF
:1077500085EE9FE28283938364827582468257829C
:10776000008711870E948018EDB7FEB73A96EDBFEB
:10777000FEBF14C000D00F92ADB7BEB71196AD9248
:10778000BC92129780E190E313968D939C9314978B
:107790000E9480180F900F900F900F902696CDBFEB
:1077A000DEBFDF91CF911F910F91FF90EF90DF909F
:1077B000CF90BF90AF909F908F907F906F905F9091
:1077C0004F903F902F900895CF93DF93EC018C81E1
:1077D0009D811816190614F40E945E0E8E819F81F9
:1077E000009711F00E949C20CE010E946647DF9115
:1077F000CF910895CF93DF93EB01E881F981309722
:1078000039F08A819B8160E070E04FEE5FEF19955F
:10781000CE010E94E43BDF91CF9108950F931F9317
:10782000CF93DF938C01DB01EA01109711F5CA01B8
:107830000E948E1F2DB73EB7285030402DBF3EBF4F
:10784000EDB7FEB73196ADB7BEB711960D931C9349
:10785000129721E430E32283338384839583C683A4
:10786000D7830E948018CDB7DEB72896CDBFDEBF84
:107870003AC02DB73EB7205130402DBF3EBFEDB7C7
:10788000FEB73196CDB7DEB789839A8381E690E360
:107890008283938315968D919C9116978459984F66
:1078A0008483958314968C91149790E00196868337
:1078B000978313968C9113978087118612968C91DB
:1078C00012978287138611968C911197848715865B
:1078D0008C91868717860E9480182DB73EB7205F4F
:1078E0003F4F2DBF3EBFDF91CF911F910F91089564
:1078F0008F929F92AF92BF92CF92DF92EF92FF92C0
:107900000F931F93CF93DF93CDB7DEB7E097CDBF33
:10791000DEBF4C018B015A01CE01019660E070E0A0
:1079200040E350E00E94EA1683E2898388E090E019
:107930000E944E477C01009709F443C081E090E02B
:1079400060E070E00E94DB0C6C01181619068CF5E3
:10795000F70100831183A282B3828483958388E830
:1079600093E160E070E04AEF5BE397010E947820CA
:10797000F701868397830097E1F0C601B4014BE7D6
:1079800050E00E94D20D8C010097B9F4C60164EA60
:107990007FE3A7010E944B0D97FD0EC0C601BE01FB
:1079A0006F5F7F4F40E350E00E946C0F97FF0BC06A
:1079B00003C00DEF1FEF01C08C01C7010E94E43B23
:1079C00002C00DEF1FEFC801E096CDBFDEBFDF9113
:1079D000CF911F910F91FF90EF90DF90CF90BF90CC
:1079E000AF909F908F900895CF92DF92EF92FF9289
:1079F0000F931F93CF93DF9300D00F92CDB7DEB7D5
:107A00007C01623071050CF440C0DA0112968D9150
:107A10009C911397BE016F5F7F4F0E940C150097DA
:107A2000A1F1CE0101966EE07CE3A7010E94783CB3
:107A30008C0197FD05C09BE8C92E90E3D92E04C0A8
:107A40008EE8C82E80E3D82EC8010E948E1FEDB7A5
:107A5000FEB73A97EDBFFEBF3196ADB7BEB71196F0
:107A6000ED92FC92129722E930E322833383C482A1
:107A7000D58206831783808791870E948018EDB78F
:107A8000FEB73A96EDBFFEBF14C000D00F92ADB75F
:107A9000BEB71196ED92FC9212978FE990E3139680
:107AA0008D939C9314970E9480180F900F900F90C5
:107AB0000F902496CDBFDEBFDF91CF911F910F9124
:107AC000FF90EF90DF90CF9008954F925F926F926A
:107AD0007F928F929F92AF92BF92CF92DF92EF925E
:107AE000FF920F931F93CF93DF93CDB7DEB7C454AC
:107AF000D040CDBFDEBF8B01DE011196E9EBF0E394
:107B000024E301900D922150E1F7DC016D917D910C
:107B10008D919C9120E831E541E050E00E941A519E
:107B20002DAB3EAB4FAB58AF20E13EE040E050E024
:107B30000E943C51F80122832CE330E040E050E009
:107B40000E943C51D80111962C9311976C936DA90A
:107B50007EA98FA998AD6C5F7F4F8F4F9F4F27E015
:107B600030E040E050E00E943C51F8016187A2EB18
:107B70004A2EA7E05A2E612C712C2BC16DA97EA92B
:107B80008FA998AD2DE631E040E050E00E943C51D5
:107B900073016201C20ED31EE41EF51EDC01CB018F
:107BA0008827B7FD83959927AA27BB27C81AD90A22
:107BB000EA0AFB0A2196CCAEDDAEEEAEFFAE21970F
:107BC00053014201089481089108A108B108A70156
:107BD0009601215030404040504025962CAF3DAF9B
:107BE0004EAF5FAF2597C501B40124E030E040E01F
:107BF00050E00E943C51DC01CB018827B7FD839502
:107C00009927AA27BB2769017A01C81AD90AEA0A63
:107C1000FB0AC9AEDAAEEBAEFCAEC501B40124E698
:107C200030E040E050E00E943C516B017C01CC24EC
:107C3000F7FCC394DD24EE24FF24C501B4012CE934
:107C40003FEF4FEF5FEF0E943C51C20ED31EE41E88
:107C5000F51E29AD3AAD4BAD5CAD2C0D3D1D4E1D55
:107C60005F1D29AF3AAF4BAF5CAFC501B40120E94E
:107C700031E040E050E00E943C51DC01CB0188271C
:107C8000B7FD83959927AA27BB2769017A01C81AEE
:107C9000D90AEA0AFB0AD701C601C9ACDAACEBACD7
:107CA000FCACC80ED91EEA1EFB1EC9AEDAAEEBAEA6
:107CB000FCAE25966CAD7DAD8EAD9FAD259720E9D0
:107CC00031E040E050E00E943C516B017C01CC244B
:107CD000F7FCC394DD24EE24FF2425966CAD7DAD26
:107CE0008EAD9FAD259720E73EEF4FEF5FEF0E94EF
:107CF0003C51C20ED31EE41EF51E25966CAD7DAD23
:107D00008EAD9FAD259724E630E040E050E00E9424
:107D10003C5149015A01DC01CB018827B7FD83950D
:107D20009927AA27BB27881A990AAA0ABB0A259667
:107D30006CAD7DAD8EAD9FAD259724E030E040E089
:107D400050E00E943C51DC01CB018827B7FD8395B0
:107D50009927AA27BB27821B930BA40BB50B880E70
:107D6000991EAA1EBB1EC80CD91CEA1CFB1CC30111
:107D7000B20121962CAD3DAD4EAD5FAD2197621B9A
:107D8000730B840B950B2DE631E040E050E00E9430
:107D9000DC50DC01CB01C80ED91EEA1EFB1E89ADEA
:107DA0009AADABADBCAD8C0D9D1DAE1DBF1DCDA85C
:107DB000DEA8EFA8F8ACC80ED91EEA1EFB1ECDAA9D
:107DC000DEAAEFAAF8AE21964CAC5DAC6EAC7FACEF
:107DD0002197CDA8DEA8EFA8F8ACF7FCCFCE23E022
:107DE000C22ED12CE12CF12CC420D520E620F72086
:107DF000C114D104E104F104E1F4C301B20124E6A9
:107E000030E040E050E00E943C51DC01CB010097A3
:107E1000A105B10599F4C301B20120E931E040E0C8
:107E200050E00E943C51DC01CB010097A105B10557
:107E300029F08DE691E0A0E0B0E004C08EE691E08C
:107E4000A0E0B0E02DA93EA94FA958AD28173907E9
:107E50004A075B070CF092CEC2018C569740D801BE
:107E600015968D939C93169717962D933C93189780
:107E7000C114D104E104F104F9F4C301B20124E610
:107E800030E040E050E00E943C51DC01CB01009723
:107E9000A105B105A1F4C301B20120E931E040E040
:107EA00050E00E943C51AB01BC0181E090E04115E3
:107EB00051056105710529F080E090E002C081E084
:107EC00090E02AE130E0829FF001839FF00D929FC5
:107ED000F00D1124EC0FFD1F79964BE050E060E0AF
:107EE00070E004C0415050406040704092918291D7
:107EF000A0E0B0E0CDA8DEA8EFA8F8ACC816D9067F
:107F0000EA06FB067CF3F8014483C81AD90AEA0A98
:107F1000FB0AD701C6018F5F838381E090E0CC5BD1
:107F2000DF4FCDBFDEBFDF91CF911F910F91FF904B
:107F3000EF90DF90CF90BF90AF909F908F907F9009
:107F40006F905F904F900895AF92BF92CF92DF9263
:107F5000EF92FF920F931F93CF93DF93CDB7DEB7CE
:107F60006097CDBFDEBF5C016B018A0140335105D4
:107F700084F1CA010E944B477C01009779F1C60148
:107F8000B701A8010E94B60EAC018017910741F518
:107F9000D70190966D917D918D919C9193974F878C
:107FA000588B0E940915DC01CB0180589E47AA4AD4
:107FB000B34889839A83AB83BC83F894CE0101963E
:107FC000BE016B5F7F4F0E94653D78944F85588955
:107FD00007C040EF5FEFEE24FF2402C04DEF5FEFDC
:107FE000D501ED91FC911197309741F012968D914A
:107FF0009C911397BE016B5F7F4F1995C7010E943B
:108000006647C5010E94E43B6096CDBFDEBFDF91AD
:10801000CF911F910F91FF90EF90DF90CF90BF9085
:10802000AF900895CF92DF92EF92FF920F931F933C
:10803000CF93DF936C018B01CB010E94F0167C0182
:10804000C0E0D0E00DC0B8016C0F7D1FA7014C1B34
:108050005D0BC6010E946C0F97FD07C0C80FD91FAA
:10806000CE15DF0584F380E090E0DF91CF911F9182
:108070000F91FF90EF90DF90CF9008958F929F9295
:10808000AF92BF92CF92DF92EF92FF920F931F9326
:10809000CF93DF934C015B016A0180E490E00E9482
:1080A0004B477C0100E010E01DC0E601C01BD10B76
:1080B000C134D10514F0C0E4D0E0B501600F711FE8
:1080C000C701AE010E94BF54C401B701AE010E94B6
:1080D0006C0FEC0197FF04C0C7010E9466470AC0FD
:1080E000080F191F0C151D0504F3C7010E946647F0
:1080F000C0E0D0E0CE01DF91CF911F910F91FF90B2
:10810000EF90DF90CF90BF90AF909F908F900895A9
:108110000F931F93CF93DF938C01EB01CB010E9450
:10812000C854AC01C801BE010E943E40DF91CF910E
:108130001F910F910895EF92FF920F931F93CF938A
:10814000DF93CDB7DEB76C97CDBFDEBF8C018EE479
:108150009FE2A1E4B0E08B879C87AD87BE87FE01DC
:108160003F968EE0DF011D928A95E9F70115110512
:1081700009F499C0C8016FE078E00E9488409C0132
:1081800097FD93C0CE01019660E070E040E050E0C2
:1081900020E030E00E940D0C009731F4CE010196F2
:1081A0000E9491167C0104C08AE0E82E81E3F82E3B
:1081B000C80160E77AE00E9488409C0197FD75C085
:1081C000C801B7010E9412409C0197FD6EC0C80112
:1081D00065E87AE00E9488409C0197FD66C0CE0168
:1081E00005960E94670C009789F58DB79EB7429758
:1081F0008DBF9EBFEDB7FEB73196CE010B96ADB7E2
:10820000BEB711968D939C93129782E190E0828382
:1082100093838EE091E3848395838D818683178297
:108220008E81808711868F818287138688858487D7
:1082300015868985868717868A85808B118A0E9494
:10824000BF558DB79EB742968DBF9EBFC80160EAED
:108250007AE00E9488409C0197FD27C0C801BE01BA
:10826000655F7F4F0E9412409C0197FD1EC0C801B0
:1082700066EB7AE00E9488409C0197FD16C0C80119
:1082800061ED7AE00E9488409C0197FD0EC0C80114
:1082900066EF7CE00E9488409C01181619062CF4B9
:1082A00020E030E002C02FEF3FEFC9016C96CDBF58
:1082B000DEBFDF91CF911F910F91FF90EF90089556
:1082C000EF92FF920F931F93CF93DF930F920F9232
:1082D000CDB7DEB78C017B016CE271E30E94FF1623
:1082E000009709F471C0C8016EE271E30E94FF16A5
:1082F000009709F469C0C80161E371E34CE050E004
:108300000E94FC16009709F058C000D000D0EDB7CD
:10831000FEB73196045F1F4FADB7BEB711960D93F0
:108320001C9312978EE391E382839383CE0101968F
:10833000848395830E94F6552DB73EB72A5F3F4F41
:108340002DBF3EBF009709F43FC089819A818330D9
:10835000910511F1843091054CF481309105B1F013
:1083600082309105B4F4009771F02EC085309105EC
:10837000C9F0853091059CF086309105B1F08730C9
:10838000910511F515C080E290E014C081E290E003
:1083900011C082E290E00EC083E290E00BC084E264
:1083A00090E008C085E290E005C086E290E002C05F
:1083B00087E290E00E94594607C0C8016BE471E370
:1083C0000E94FF16009729F4C7010E949B409C0160
:1083D00028C0C80167E571E30E94FF16009781F489
:1083E000C70164EF71E00E9488409C0197FD19C0AD
:1083F000C70160E372E045EE54E00E943E4008C0D1
:10840000E114F10461F0C70165E177E00E94884062
:108410009C01181619062CF420E030E002C02FEF62
:108420003FEFC9010F900F90DF91CF911F910F91F6
:10843000FF90EF9008950F931F93CF938C01C62F59
:10844000BA0180E090E026E631E040E050E00E9492
:10845000DC5020914C3330914D3340E050E00E948D
:108460001A5120934A3330934B332FB7F894F801C5
:10847000308181E090E002C0880F991FCA95E2F731
:10848000880F880F832B80832FBFCF911F910F916F
:1084900008950F931F93CF93DF93CDB7DEB72A973D
:1084A000CDBFDEBFBE016C5F7F4F87E0FB01119245
:1084B0008A95E9F78E010F5F1F4F83E0F801119253
:1084C0008A95E9F786E0888781E08E8380E092E0F4
:1084D0000E94075080E092E06BE172E40E946449E0
:1084E00019821A828B81807F81608B8380E092E089
:1084F00060E0A8010E946C5082E06FE270E00E9490
:108500003E47182F00E082E06EE270E00E943E4796
:1085100090E0802B912B80934C3390934D3380E0EF
:1085200092E00E94BF499FB7F894E0E0F2E08081BA
:10853000846080839FBF2A96CDBFDEBFDF91CF913D
:108540001F910F91089580914A3390914B3381513F
:108550009140089500D000D0EDB7FEB73196ADB789
:10856000BEB711968D939C93129781E691E3828317
:108570009383648375830E9480188DB79EB7069697
:108580008DBF9EBF08950E9454460E94B620089554
:108590006115710529F08FB7F894809350330895D1
:1085A000809150338FBF0895662349F000D00F9219
:1085B000EDB7FEB78183928383E791E308C000D0D3
:1085C0000F92EDB7FEB7818392838FE891E38383A7
:1085D00094830E9480180F900F900F900F90089531
:1085E000CF93DF93EC01CB010097A9F400D00F9259
:1085F000ADB7BEB71196CD93DC93129789EA91E39C
:1086000013968D939C9314970E9480180F900F904F
:108610000F900F901AC00E94911600D000D0EDB7B5
:10862000FEB73196ADB7BEB71196CD93DC931297D6
:108630002BEB31E322833383848395830E9480185C
:10864000EDB7FEB73696EDBFFEBFDF91CF9108952F
:10865000AF92BF92CF92DF92EF92FF920F931F9350
:10866000CF93DF93CDB7DEB7CB56D040CDBFDEBFC3
:108670001A820E94704680E490E063EC72E40E94EB
:108680002B460E94A21F97FDCAC180EA99E040E0F4
:1086900052EC61E070E028E030E000E010E0E1E062
:1086A000EE2EF12CCC24DD240E94204597FDB7C18D
:1086B00080E090E063EB75E440EA59E024E030E0CC
:1086C0000E94811D5C01009709F4A9C10E947D22CE
:1086D00080EA9BE040E052EC61E070E028E030E0AE
:1086E0000E94204597FD9BC180E090E06CE975E415
:1086F00043EB55E428EC32E400EA1BE00E94230A35
:1087000097FD8DC180EA9BE080934E3390934F3369
:108710000E944942CE0102960E945D0ACE01019656
:108720000E948F138AEA92E4B5010E94550B80EFF4
:1087300092E4B5010E945E0C84ED92E4B5010E94C2
:108740007B14C5016FE272E340E050E00E946718BD
:10875000C50163EE72E340E050E00E946718C50176
:108760006BEF72E340E050E00E946718C50165EFCF
:1087700072E340E050E00E946718C50169EB72E3C4
:1087800040E050E00E946718C50163EB72E340E0EF
:1087900050E00E946718C50169EE72E3AE01445DC6
:1087A0005F4F0E946718C5016FEE72E3AE01445D32
:1087B0005F4F0E946718C5016DEA72E340E050E028
:1087C0000E946718C50167EA72E340E050E00E942A
:1087D0006718C50161EA72E340E050E00E94671843
:1087E000C5016BE972E340E050E00E946718C501E3
:1087F00065E972E340E050E00E946718C5016FE54B
:1088000072E340E050E00E946718C5016FE872E330
:1088100040E050E00E946718C50169E872E340E05B
:1088200050E00E946718C50163E872E340E050E041
:108830000E946718C5016DE772E340E050E00E94B6
:108840006718C50167E772E340E050E00E946718CF
:10885000C50161E772E340E050E00E946718C5017E
:108860006BE672E340E050E00E946718C50165E6E0
:1088700072E340E050E00E946718C50163E572E3CF
:1088800040E050E00E946718C5016DE472E340E0EB
:1088900050E00E946718C50167E472E340E050E0D1
:1088A0000E946718C5016DED72E340E050E00E9440
:1088B0006718C50167ED72E340E050E00E94671859
:1088C000C50161ED72E340E050E00E946718C50108
:1088D0006BEC72E340E050E00E946718C5016FEB5B
:1088E00072E340E050E00E946718C50161E073E365
:1088F00040E050E00E946718C50169E572E340E07E
:1089000050E00E946718C50161E472E340E050E066
:108910000E946718C5016BE372E340E050E00E94DB
:108920006718C50165E372E340E050E00E946718F4
:10893000C50163E173E340E050E00E946718C501A0
:1089400069E173E340E050E00E946718C5016DE003
:1089500073E340E050E00E946718C5016DEF71E3DA
:1089600040E050E00E94671889818823B1F566E1F4
:1089700072E088EA90EC0E94DE14DC01CB018F8368
:108980009887A987BA8760E07FEF8FEF9FEF0E94FB
:10899000DE14DC01CB018B839C83AD83BE83CE01CF
:1089A0000B966BEC71E30E9402178BEC91E30E9433
:1089B000F0168BA7CE010B9666ED71E340E050E018
:1089C0000E949C0BCE010796BE016D5F7F4F40E079
:1089D00050E020E030E00E94040C80E590E00E942E
:1089E000F43380EA99E00E94D845009751F080EA7C
:1089F00099E060E070E00E948445682FC5010E9404
:108A0000E11A8A8180FF06C08DE290E00E94F9465B
:108A1000009711F40E94BD100E940121E2CF8FEF58
:108A20009FEFC559DF4FCDBFDEBFDF91CF911F91C3
:108A30000F91FF90EF90DF90CF90BF90AF9008958F
:108A4000AF92BF92CF92DF92EF92FF920F931F935C
:108A5000CF935C01C114D10409F044C026503040CA
:108A60002430310528F4215E3C4CF901C08101C05D
:108A7000C0E00130110539F00130110538F0023045
:108A8000110581F502C0C06201C0C063F2E0EF16BB
:108A9000F10409F4C8609A01AB0184E0220F331F8E
:108AA000441F551F8A95D1F7213088E4380788EE96
:108AB000480781E0580750F460E078E488EE91E0E0
:108AC0000E941A512150304088E103C02FEF3FEF40
:108AD0008CE1F5011482C58326833783848380E08B
:108AE00090E002C086EF9FEFCF911F910F91FF9012
:108AF000EF90DF90CF90BF90AF900895FC018181FF
:108B000085FFFDCF608308950F931F93CF93DF936D
:108B1000EC018B010E94AF200115110531F4898110
:108B200087FFFDCF888190E002C086EF9FEFDF9145
:108B3000CF911F910F910895DC0180E090E00EC06D
:108B400011962C91119727FFFBCF2C916115710580
:108B500021F0FB01E80FF91F208301968417950788
:108B60007CF3CA010895CF92DF92EF92FF920F93A8
:108B70001F93CF93DF936C017A018B01C0E0D0E0AB
:108B80000AC0F80161918F01772767FD7095C601D2
:108B90000E947E452196CE15DF059CF3C701DF912B
:108BA000CF911F910F91FF90EF90DF90CF9008959C
:108BB000FC01818190E08078907008958530910566
:108BC00040F4FC01EE0FFF1FED5DFC4C80819181B4
:108BD000089584EE91E30895CF92DF92EF92FF9291
:108BE0006B017C01E0915133F0915233309709F0E1
:108BF00019958091533390915433A0915533B0918E
:108C000056338C0D9D1DAE1DBF1DBC01CD010E94B4
:108C10009B48FF90EF90DF90CF900895809357335B
:108C2000909358339C01B901882777FD8095982F40
:108C300028EE33E040E050E00E94DC500E941A51E0
:108C400020935333309354334093553350935633DA
:108C500080E090E00895CF92DF92EF92FF926C0156
:108C600060935133709352330E94BB488CEE95E46D
:108C70000E94B648C6010E940E46C0905333D09061
:108C80005433E0905533F09056330E9476486C0D83
:108C90007D1D8E1D9F1D0E949B4880E090E0FF90EF
:108CA000EF90DF90CF900895809157339091583393
:108CB0000895CF93DF93EC010E94F946009721F0CD
:108CC000CE010E94294703C0CE010E941447DF91C4
:108CD000CF9108950E94144708950E94294708954E
:108CE00087E0E0EAF0E082830E9496470E94ED4729
:108CF00080EA96E068E043E050E00E94694780EA3D
:108D000096E064E040E050E00E94694783E090E034
:108D100060E10E94BF4784E090E060E10E94BF47AD
:108D200086E090E060E10E94BF47789480E090E0A8
:108D300008959C0108C08FE39FE10197F1F700C0FF
:108D400000002150304021153105A9F70895CF9337
:108D5000C82F8A3031F480EA99E06DE070E00E941B
:108D60007E456C2F772767FD709580EA99E00E9419
:108D70007E45CF91089589E593E3089580E090E0E2
:108D8000089560FF18C0282F26952695269530E077
:108D9000205D3F4F877061E070E002C0660F771F73
:108DA0008A95E2F7C90155E0880F991F5A95E1F7B6
:108DB00040E050E019C061FF19C0282F2695269584
:108DC000269530E0205D3F4F877061E070E002C083
:108DD000660F771F8A95E2F7C90145E0880F991F52
:108DE0004A95E1F741E050E00E94694780E090E059
:108DF0000895E82FE695E695E695F0E0F09665E0B3
:108E0000EE0FFF1F6A95E1F74085877021E030E0A3
:108E100002C0220F331F8A95E2F7422381E090E0DF
:108E200011F480E090E00895E82FE695E695E69548
:108E3000F0E0F09675E0EE0FFF1F7A95E1F787708E
:108E400021E030E002C0220F331F8A95E2F725832C
:108E50000895E82FE695E695E695F0E0F096A5E012
:108E6000EE0FFF1FAA95E1F7877021E030E002C006
:108E7000220F331F8A95E2F7268308954091CA0195
:108E8000E62FF72F8093CA0184914093CA01089579
:108E900080E090E008950E946B5108950F931F9316
:108EA000CF93DF938C010E946B51EC01009729F066
:108EB00060E070E0A8010E94EA16CE01DF91CF9138
:108EC0001F910F9108950E949A5208950E94015295
:108ED0000895CF93DF93DC0180E090E0C62FD0E0CF
:108EE0009E01082E02C0359527950A94E2F720FFCF
:108EF00004C0FD01E80FF91F508B019688309105E1
:108F000079F740FF0DC041FF04C015966C9315978B
:108F100003C016966C93169711966C93119703C025
:108F200012966C931297DF91CF9108958FEF8093F3
:108F3000700080937100809372008093730080931F
:108F4000740080937500809376009FB7F8948091A9
:108F500050008260809350009FBF8091510081FF3C
:108F6000FCCF80E490E061E00E945E499FB7F894F6
:108F7000809150008E7F809350009FBF0895FC0128
:108F80009FB7F894E059FF4F6095808186238083D6
:108F90009FBF0895FC019FB7F894E059FF4F80816F
:108FA000862B80839FBF0895AB01282F2695269599
:108FB000269530E0205D3F4F877061E070E002C091
:108FC000660F771F8A95E2F7C90175E0880F991F30
:108FD0007A95E1F70E946947089580E263E070E0C6
:108FE0000E94D44781E263E070E00E94D44782E2AD
:108FF00063E070E00E94D44783E263E070E00E9487
:10900000D44784E263E070E00E94D44785E263E0E5
:1090100070E00E94D44786E263E070E00E94D4478B
:1090200087E263E070E00E94D44788E160E078E185
:109030000E94D44789E160E078E10E94D4478AE148
:1090400060E078E10E94D4478BE160E078E10E9423
:10905000D4478CE160E078E10E94D4478DE160E084
:1090600078E10E94D44788E760E078E10E94D44725
:1090700089E760E078E10E94D44788E060E077E02B
:109080000E94D4478BE061E070E00E94D44783E106
:1090900063E070E00E94D44782E160E070E00E94EB
:1090A000D4478BE163E070E00E94D4478AE160E03E
:1090B00070E00E94D44708959091020481E092FDEF
:1090C00080E00895DC01CB0110920004209101049E
:1090D00020FDFCCFE0E0F4E080879187A093153479
:1090E000B093163481E08093000408950F931F938A
:1090F0002FB7F8940091153410911634809108041C
:1091000090910904009731F43091030430FF02C0BC
:109110000F5F1F4F2FBF20E030E09801112700277D
:10912000A0E0B0E0082B192B2A2B3B2BB801C9017A
:109130001F910F910895DC01CB01E0E0F4E021E004
:109140002283848795878093193490931A34A0934F
:109150001734B0931834E0E0F4E08091010480FD0E
:10916000FACF82E0838385E08283089580931B3465
:1091700090931C34089580E090E064E00E94BF4723
:1091800021E0E0E4F0E02383E0E0F4E08FEF9FEF04
:1091900082879387108611862283208308951F92E9
:1091A0000F920FB60F9208B60F9211248F939F93D0
:1091B00080911534909116340196809315349093D4
:1091C00016349F918F910F9008BE0F900FBE0F9095
:1091D0001F9018951F920F920FB60F9208B60F921C
:1091E00009B60F920BB60F9211240F931F932F9372
:1091F0003F934F935F936F937F938F939F93AF931F
:10920000BF93EF93FF930091153410911634409162
:1092100017345091183404171507B8F181E0E0E0D5
:10922000F4E08283E0911B34F0911C34309769F1B3
:10923000809108049091090420E030E09801112702
:109240000027A0E0B0E0082B192B2A2B3B2BCA01EA
:10925000A0E0B0E0DC0199278827409119345091B3
:109260001A3460E070E0842B952BA62BB72B801767
:109270009107A207B30730F08C019D010F5F1F4FCC
:109280002F4F3F4FC901B8011995FF91EF91BF9141
:10929000AF919F918F917F916F915F914F913F918E
:1092A0002F911F910F910F900BBE0F9009BE0F9041
:1092B00008BE0F900FBE0F901F9018951BBEFC01AB
:1092C00028ED24BF608308952FB7F89432E08030F2
:1092D000930729F460931F347093203408C032E060
:1092E0008034930721F460931D3470931E342FBF94
:1092F000089522E08030920771F480915933982FBD
:109300009F5F909359338823B9F481E090E062E045
:109310000E94BF47089522E08034920769F480914B
:109320005A33982F9F5F90935A33882329F482E011
:1093300090E062E00E94BF47089522E080309207EB
:1093400069F4809159338150809359338823B1F463
:1093500081E090E062E00E94CA47089522E08034F4
:10936000920761F480915A33815080935A33882355
:1093700029F482E090E062E00E94CA4708951F93BA
:10938000CF93DF93EC011FB7F8940E94794988814D
:10939000816088831FBFDF91CF911F910895CF9384
:1093A000CFB7F894FC0120812E7F20830E949D4935
:1093B000CFBFCF91089522E08030920721F481E061
:1093C0009091593307C022E08034920739F481E04C
:1093D00090915A33992319F480E0089580E008951C
:1093E0008091CF0187FDFCCF08951F93CF93DF932A
:1093F000C0ECD1E01A858A878BEC91E061E00E9495
:109400005E491A87DF91CF911F910895682F82E0FE
:1094100070E00E943E470895CF93DF93EC0188E00F
:109420000E94064A888389E00E94064A89838AE06E
:109430000E94064A8A838BE00E94064A8B838CE056
:109440000E94064A8C838DE00E94064A8D8380E14B
:109450000E94064A8E8382E10E94064A8F8383E13E
:109460000E94064A888784E10E94064A898785E12E
:109470000E94064A8A87DF91CF9108950F931F9328
:10948000CF93DF930F920F92CDB7DEB789839A8384
:109490000E94F04900EC11E0F80112829A81918358
:1094A0008981808386E090E00E94F549F8018481FB
:1094B0000F900F90DF91CF911F910F910895EF9230
:1094C000FF920F931F93CF93DF9300D00F92CDB7EE
:1094D000DEB77C01CB014B835C8369839A830E9456
:1094E000F0490CEC11E0F801208128602083B701DD
:1094F0006050704F89819A814B815C810E94E35456
:10950000F8018081877F80832496CDBFDEBFDF9105
:10951000CF911F910F91FF90EF9008950E94F04915
:109520008091CF0181FF09C086E3E0ECF1E0828702
:109530008BEC91E061E00E945E490895EF92FF920A
:109540001F93CF93DF9300D0CDB7DEB720ECE22E90
:1095500021E0F22EF701128569838A839B830E94A2
:109560008E4A0E94F04923E3F701228712829B81F1
:1095700091838A8180836981648385E382878BEC10
:1095800091E061E00E945E49F70112872396CDBF0A
:10959000DEBFDF91CF911F91FF90EF900895EF9282
:1095A000FF921F93CF93DF930F920F92CDB7DEB749
:1095B00030ECE32E31E0F32EF70112856A838983C4
:1095C0000E94F04993E3F701928712821182898108
:1095D00080836A81648312870F900F90DF91CF910F
:1095E0001F91FF90EF900895FF920F931F93CF93D9
:1095F000DF93EC0100EC11E0F090CA010E94F04909
:1096000083E3F80182871282118280E08093C00197
:10961000999194838F5F8032C9F7E0ECF1E0F28694
:10962000DF91CF911F910F91FF900895CF93DF931A
:109630000F92CDB7DEB789830E94F049898190E00F
:1096400045E0880F991F4A95E1F7E0ECF1E01282BE
:109650009183808385E390E00E94F5490F90DF912C
:10966000CF910895CF92DF92EF92FF920F931F93C5
:10967000CF93DF938C016B017A012BC0C8018F71EE
:1096800090700097D1F480E2E816F104B0F0C601C2
:109690000E94F44AC80155E0969587955A95E1F7DE
:1096A0000E94164B005E1F4FE0E2F0E0CE0EDF1E80
:1096B00080EE9FEFE80EF91E0CC0E8012196C8016C
:1096C000F60161916F010E949E4A0894E108F10839
:1096D0008E01E114F10491F6DF91CF911F910F916A
:1096E000FF90EF90DF90CF900895CF93DF930F928C
:1096F000CDB7DEB789830E94F049898190E065E0AB
:10970000880F991F6A95E1F7E0ECF1E012829183EE
:10971000808384E390E00E94F5490F90DF91CF9120
:109720000895EF92FF921F93CF93DF930F92CDB7DF
:10973000DEB770ECE72E71E0F72E1091CA01898335
:109740000E948E4A0E94F04993E3D7011A969C9397
:109750001A9712961C92129711961C92119790E0EC
:10976000E0ECF1E089819093C00184839F5F9032A7
:10977000D1F7E0ECF1E012870F90DF91CF911F91CC
:10978000FF90EF900895CF93DF930F92CDB7DEB7A0
:1097900089830E94F049898190E0E5E0880F991F54
:1097A000EA95E1F7E0ECF1E012829183808382E3B5
:1097B00090E00E94F5490F90DF91CF910895CF93EB
:1097C000C82F8FEF0E94914B8C2F0E94C34BCF91DB
:1097D00008950E94F04980E390E00E94F5490895C1
:1097E0008FEF0E94914B0E94E94B0895CF92DF9238
:1097F000EF92FF921F93CF93DF936B017C01DA010D
:10980000C901C0ECD1E01A852AE32A87C8827727EC
:109810006F2D5E2D4D2D49836701EE24FF24CA82F2
:109820008C83492F5A2F6B2F77274D83CD01AA2781
:10983000BB278E838BEC91E061E00E945E491A8722
:10984000DF91CF911F91FF90EF90DF90CF9008951F
:10985000CF92DF92EF92FF920F931F93CF93DF93FC
:109860000F920F92CDB7DEB7F82EE92E8A0169016B
:1098700069837A830E94F0496981862F7A81972FC4
:10988000AF2DBE2D0EC00BB6ABBFFC0127910BBE9A
:10989000F80121938F010196A11DB11D0894C10803
:1098A000D108C114D10479F70F900F90DF91CF91B7
:1098B0001F910F91FF90EF90DF90CF900895EF925E
:1098C000FF920F931F93CF93DF93DC01CB017A01BB
:1098D0008901EC01D1700AC081E0BE010E943E47BF
:1098E000F70181937F012196015010400115110568
:1098F00099F7DF91CF911F910F91FF90EF9008950D
:109900002F923F924F925F926F927F928F929F928F
:10991000AF92BF92CF92DF92EF92FF920F931F937D
:10992000CF93DF930F920F92CDB7DEB7DC01CB015F
:109930002A017901702E8C01662457C061E0C62E81
:10994000D12C8824992454011401772089F081E0D6
:10995000B4010E943E47898381E0B6010E943E47E0
:109960008A8389819A812FEF8F3F920731F407C054
:109970008FEF9FEF89839A8302C066246394E1147A
:10998000F104D9F00215130561F40894E108F10817
:109990000F5F1F4FD2018D912D018983E114F104D6
:1099A00061F00C151D0549F40894E108F1080F5FFA
:1099B0001F4FF20181912F018A8349815A81C5018C
:1099C000B4010E948B0782E090E0A0E0B0E0880E36
:1099D000991EAA1EBB1EA2E0B0E0CA0EDB1EB1E0BB
:1099E000CB16B2E0DB0609F0AFCFE114F10409F0C9
:1099F000A5CF662041F00E94F04960E070E0CB0105
:109A000048E10E947C070E94F04960E070E0CB01D1
:109A10004AE10E947C070F900F90DF91CF911F9138
:109A20000F91FF90EF90DF90CF90BF90AF909F90FD
:109A30008F907F906F905F904F903F902F90089500
:109A40002F923F924F925F926F927F928F929F924E
:109A5000AF92BF92CF92DF92EF92FF920F931F933C
:109A6000CF93DF9300D000D0CDB7DEB7DC01CB01C0
:109A70004B835C831901412CEEEF5E2EEFEF6E2ECF
:109A8000EFEF7E2E482259226A227B226C017D0153
:109A90007AC00E94F0495301420120E031E010E019
:109AA000002369F00BB6ABBEF401879196910BBE13
:109AB00089839A834FEF8F3F940731F406C08FEF6D
:109AC0009FEF89839A8301C011E02114310471F161
:109AD000C814D904EA04FB0489F408942108310865
:109AE0000894C11CD11CE11CF11CAB81BC818D917F
:109AF000AB83BC83898321143104C1F0D501C40137
:109B00000196A11DB11DC816D906EA06FB0671F41F
:109B10000894210831080894C11CD11CE11CF11CD7
:109B2000EB81FC818191EB83FC838A8349815A819B
:109B3000C501B4012D833E830E948B0782E090E033
:109B4000A0E0B0E0880E991EAA1EBB1E2D813E81AA
:109B50002150304009F0A4CF112331F00E94F04988
:109B6000C301B20145E205C00E94F049C301B20140
:109B700044E20E947C0780E092E0A0E0B0E0480E62
:109B8000591E6A1E7B1E2114310409F082CF2696CD
:109B9000CDBFDEBFDF91CF911F910F91FF90EF906E
:109BA000DF90CF90BF90AF909F908F907F906F90FD
:109BB0005F904F903F902F9008950F931F93CF93F6
:109BC000DF930F92CDB7DEB789830E94F04900EC96
:109BD00011E08981F801808387E090E00E94F549D7
:109BE000F80184810F90DF91CF911F910F9108951B
:109BF000CF93DF9381309105C1F08130910520F042
:109C00008230910579F51DC082E061E270E00E942A
:109C10003E47C82F82E060E270E00E943E473C2F42
:109C200020E090E0822B932B1FC082E065E270E081
:109C30000E943E47D82F80E0C82F82E064E270E0A7
:109C40000BC082E06FE270E00E943E47D82F80E0B8
:109C5000C82F82E06EE270E00E943E4790E08C2BBD
:109C60009D2B02C080E090E0DF91CF9108951F927C
:109C70000F920FB60F9208B60F9209B60F920BB65D
:109C80000F9211242F933F934F935F936F937F9382
:109C90008F939F93AF93BF93EF93FF93E0E0F2E036
:109CA00044A155A1E0911F34F091203480E092E06E
:109CB00061E01995FF91EF91BF91AF919F918F91C5
:109CC0007F916F915F914F913F912F910F900BBEBC
:109CD0000F9009BE0F9008BE0F900FBE0F901F90FF
:109CE00018951F920F920FB60F9208B60F9209B6F1
:109CF0000F920BB60F9211242F933F934F935F93C4
:109D00006F937F938F939F93AF93BF93EF93FF9343
:109D1000E0E0F2E044A555A5E0911F34F091203435
:109D200080E092E062E01995FF91EF91BF91AF91D1
:109D30009F918F917F916F915F914F913F912F9163
:109D40000F900BBE0F9009BE0F9008BE0F900FBE74
:109D50000F901F9018951F920F920FB60F9208B692
:109D60000F9209B60F920BB60F9211242F933F93C7
:109D70004F935F936F937F938F939F93AF93BF9313
:109D8000EF93FF93E0E0F2E044A955A9E0911F347E
:109D9000F091203480E092E064E01995FF91EF911A
:109DA000BF91AF919F918F917F916F915F914F91F3
:109DB0003F912F910F900BBE0F9009BE0F9008BEE0
:109DC0000F900FBE0F901F9018951F920F920FB615
:109DD0000F9208B60F9209B60F920BB60F9211248C
:109DE0002F933F934F935F936F937F938F939F93A3
:109DF000AF93BF93EF93FF93E0E0F2E044AD55AD36
:109E0000E0911F34F091203480E092E068E01995F1
:109E1000FF91EF91BF91AF919F918F917F916F9142
:109E20005F914F913F912F910F900BBE0F9009BE04
:109E30000F9008BE0F900FBE0F901F9018951F92A5
:109E40000F920FB60F9208B60F9209B60F920BB68B
:109E50000F9211242F933F934F935F936F937F93B0
:109E60008F939F93AF93BF93EF93FF93E0E4F2E060
:109E700044A155A1E0911D34F0911E3480E492E09C
:109E800061E01995FF91EF91BF91AF919F918F91F3
:109E90007F916F915F914F913F912F910F900BBEEA
:109EA0000F9009BE0F9008BE0F900FBE0F901F902D
:109EB00018951F920F920FB60F9208B60F9209B61F
:109EC0000F920BB60F9211242F933F934F935F93F2
:109ED0006F937F938F939F93AF93BF93EF93FF9372
:109EE000E0E4F2E044A555A5E0911D34F0911E3464
:109EF00080E492E062E01995FF91EF91BF91AF91FC
:109F00009F918F917F916F915F914F913F912F9191
:109F10000F900BBE0F9009BE0F9008BE0F900FBEA2
:109F20000F901F9018951F920F920FB60F9208B6C0
:109F30000F9209B60F920BB60F9211242F933F93F5
:109F40004F935F936F937F938F939F93AF93BF9341
:109F5000EF93FF93E0E4F2E044A955A9E0911D34AA
:109F6000F0911E3480E492E064E01995FF91EF9146
:109F7000BF91AF919F918F917F916F915F914F9121
:109F80003F912F910F900BBE0F9009BE0F9008BE0E
:109F90000F900FBE0F901F9018951F920F920FB643
:109FA0000F9208B60F9209B60F920BB60F921124BA
:109FB0002F933F934F935F936F937F938F939F93D1
:109FC000AF93BF93EF93FF93E0E4F2E044AD55AD60
:109FD000E0911D34F0911E3480E492E068E0199520
:109FE000FF91EF91BF91AF919F918F917F916F9171
:109FF0005F914F913F912F910F900BBE0F9009BE33
:10A000000F9008BE0F900FBE0F901F901895DF9213
:10A01000EF92FF920F931F93CF93DF93EC018B018D
:10A0200082E0C030D80719F480E090E006C0E2E09A
:10A03000C034DE0721F581E090E00E94F84D7C01FC
:10A04000DFB6F894CE010E947949288182E08883A6
:10A05000EC86FD86F80185819681888F998F8281B3
:10A060008A8384818C8383818B838181898321701E
:10A070008081282B2883CE010E949D49DFBEDF917D
:10A08000CF911F910F91FF90EF90DF900895FF9275
:10A090000F931F93CF93DF93EC018B01FFB6F894DE
:10A0A0000E9479498881807CF8018083888D998D10
:10A0B000858396838A8182838C8184838B81838349
:10A0C00089818183CE010E949D49FFBEDF91CF919E
:10A0D0001F910F91FF900895DF92EF92FF920F93DF
:10A0E0001F93CF93DF937C018A01862F90E08370CA
:10A0F0009070009721F46695669582E001C080E03B
:10A1000060FF8F5FE701A09690E023E0880F991F22
:10A110002A95E1F7C80FD91FDFB6F894C7010E944E
:10A120007949F8018081888382818A83818189834A
:10A13000C7010E949D49DFBEDF91CF911F910F9112
:10A14000FF90EF90DF900895DF92EF92FF920F93D0
:10A150001F93CF93DF937C018A01862F90E0837059
:10A160009070009721F46695669582E001C080E0CA
:10A1700060FF8F5FE701A09690E033E0880F991FA2
:10A180003A95E1F7C80FD91FDFB6F894C7010E94CE
:10A1900079498881F80180838A81828389818183DA
:10A1A000C7010E949D49DFBEDF91CF911F910F91A2
:10A1B000FF90EF90DF900895629FD001739FF001B0
:10A1C000829FE00DF11D649FE00DF11D929FF00D47
:10A1D000839FF00D749FF00D659FF00D9927729F7E
:10A1E000B00DE11DF91F639FB00DE11DF91FBD0109
:10A1F000CF0111240895991B79E004C0991F961787
:10A2000008F0961B881F7A95C9F78095089597FBEB
:10A21000092E07260AD077FD04D049D006D00020A9
:10A220001AF4709561957F4F0895F6F79095819592
:10A230009F4F0895A1E21A2EAA1BBB1BFD010DC062
:10A24000AA1FBB1FEE1FFF1FA217B307E407F507E6
:10A2500020F0A21BB30BE40BF50B661F771F881FC2
:10A26000991F1A9469F760957095809590959B0158
:10A27000AC01BD01CF01089597FB092E05260ED034
:10A2800057FD04D0D7DF0AD0001C38F45095409514
:10A29000309521953F4F4F4F5F4F0895F6F79095BA
:10A2A0008095709561957F4F8F4F9F4F0895AA1BA2
:10A2B000BB1B51E107C0AA1FBB1FA617B70710F0B1
:10A2C000A61BB70B881F991F5A95A9F780959095E3
:10A2D000BC01CD010895CF93DF93AC01823091058D
:10A2E00010F442E050E0E0912334F091243420E077
:10A2F00030E0A0E0B0E024C0808191818417950710
:10A30000D0F08417950771F482819381109729F01A
:10A3100012968D939C9313972CC080932334909323
:10A32000243427C02115310519F08217930718F43A
:10A330009C01BD01EF0192818381DF01E92FF82F9C
:10A340003097D1F621153105F9F0C901841B950B21
:10A350008430910580F48A819B816115710521F01B
:10A36000FB018283938304C080932334909324342D
:10A37000FE01329642C0FE01E80FF91F419351934E
:10A3800002978883998339C0809121349091223437
:10A39000009741F48091F1319091F2318093213412
:10A3A000909322342091EF313091F0312115310515
:10A3B00041F42DB73EB78091F3319091F431281BD1
:10A3C000390BE0912134F0912234E217F30798F42D
:10A3D0002E1B3F0B2417350770F0CA010296281771
:10A3E000390748F08E0F9F1F8093213490932234B9
:10A3F0004193519302C0E0E0F0E0CF01DF91CF91B3
:10A4000008950F931F93CF93DF939C01009709F456
:10A410008CC0DC01129712961D921C9213976091CA
:10A420002334709124346115710589F48D919C91C8
:10A430001197820F931F20912134309122342817D5
:10A44000390769F5A0932134B09322346EC0FB0123
:10A4500040E050E001C0FC01EA17FB0730F48281C4
:10A460009381AF010097B9F71FC0E9012297EA83F2
:10A47000FB8308811981C901800F911F8E179F07E7
:10A4800059F480819181800F911F0296888399836E
:10A49000828193818A839B834115510529F4A0937E
:10A4A0002334B093243441C0FA01A283B383C19111
:10A4B000D191EC0FFD1FAE17BF0781F4F901929106
:10A4C00082918C0F9D1F0296DA018D939C931197B8
:10A4D0008281938112968D939C931397E0E0F0E034
:10A4E00002C0FB01BC01DB0112968D919C91139778
:10A4F0000097B9F7CB0102962D913C911197820FED
:10A50000931F20912134309122342817390769F4A0
:10A51000309729F4109223341092243402C012820E
:10A5200013826093213470932234DF91CF911F9175
:10A530000F9108958F929F92AF92BF92CF92DF9228
:10A54000EF92FF920F931F93CF93DF930F920F928F
:10A55000CDB7DEB78C01009729F4CB010E946B5177
:10A560008C01B8C0DC01A60FB71FFC013297AE17F3
:10A57000BF0708F4ADC02081318126173707B0F03E
:10A580002530310508F4A6C0C9010497861797073E
:10A5900008F4A0C022503040261B370B2D933D936A
:10A5A000CD01608371830E94015294C06B01C21A75
:10A5B000D30A5C01A20EB31EE0912334F09124343F
:10A5C00040E050E08824992449C0EA15FB05E1F5F4
:10A5D000E080F180C70102968C159D05A8F1A701C6
:10A5E0004C195D09CA0102960F2EFEEFCF2EFFEF28
:10A5F000DF2EF02DC00ED11E8530910578F08281BE
:10A60000938112968D939C9313974D935C9311971E
:10A61000F601608371839A2F8B2F0AC0C9010296BD
:10A620008E0D9F1DD6018D939C93119792818381EE
:10A630008114910421F0F401928383834BC09093A1
:10A6400023348093243446C0808191814817590770
:10A6500008F4AC01828193814F01FC01309709F02D
:10A66000B4CF80912134909122348A159B05E9F46E
:10A6700046175707D0F48091EF319091F031009751
:10A6800041F48DB79EB72091F3313091F431821BA4
:10A69000930BA817B907E0F4A0932134B0932234A8
:10A6A000F80132976083718315C0CB0129833A8307
:10A6B0000E946B517C0129813A81009749F0B801D1
:10A6C000A9010E94E354C8010E940152870102C0FF
:10A6D00000E010E0C8010F900F90DF91CF911F9123
:10A6E0000F91FF90EF90DF90CF90BF90AF909F9031
:10A6F0008F9008952F923F924F925F926F927F9228
:10A700008F929F92BF92CF92DF92EF92FF920F9320
:10A710001F93CF93DF933B018A016115710519F0F7
:10A72000FB01808391830115110539F098012250B6
:10A7300030402332310508F003C16C0176010894E2
:10A74000C11CD11CF701C08146018C2F90E00E94F2
:10A75000B754009799F7CD3249F4F701C181B2E0BF
:10A760008B2E912C8E0C9F1CD1E00AC0CB3239F479
:10A77000F701C181A2E08A2E912C8E0C9F1CD0E0A3
:10A780000115110519F000311105C1F4C03381F430
:10A79000F4018081883711F0883551F4F401C181CA
:10A7A00082E090E0880E991ED26000E110E006C0C1
:10A7B0000115110519F4C033C1F422C00830110588
:10A7C000F9F00930110524F40230110509F507C02C
:10A7D0000A30110551F000311105D1F427C0C12C08
:10A7E000D12CE12C70E4F72E26C00AE010E06CECCE
:10A7F000C62E6CECD62E6CECE62E6CE0F62E1BC052
:10A8000008E010E0C12CD12CE12C50E1F52E13C052
:10A810009801442737FD4095542F60E070E080E0B8
:10A8200090E80E941A5169017A0105C0C12CD12C0F
:10A83000E12C48E0F42E20E040E050E0BA0118019D
:10A84000442437FC4094542C30EDB32EBC0E99E0D8
:10A850009B1570F48C2F81548A3118F499ECB92E21
:10A8600006C08C2F81568A3150F589EAB82EBC0E6D
:10A870008B2D90E08017910714F527FD1CC0C4169E
:10A88000D506E606F706A0F0CB01BA01A2019101B8
:10A890000E94DC50AB01BC014B0D511D611D711DAF
:10A8A0004130E0E05E07E0E06E07E0E87E0710F090
:10A8B0002FEF01C021E0F401C1914F01C5CF611418
:10A8C000710489F0222339F0089481089108F3017A
:10A8D0008082918208C0D1FF1AC0C4010297F3019F
:10A8E0008083918314C027FF12C0D0FF05C040E0D1
:10A8F00050E060E070E804C04FEF5FEF6FEF7FE77C
:10A9000082E290E0809325349093263416C0D0FFE5
:10A9100008C070956095509541955F4F6F4F7F4F80
:10A920000CC077FF0AC082E290E0809325349093B8
:10A9300026344FEF5FEF6FEF7FE78A019B0103C083
:10A9400000E010E09801B801C901DF91CF911F919B
:10A950000F91FF90EF90DF90CF90BF909F908F90DE
:10A960007F906F905F904F903F902F90089591113E
:10A9700057C6803219F089508550D0F70895FB01F1
:10A98000DC0102C005900D9241505040D8F7089567
:10A99000FC0105900020E9F7809590958E0F9F1F90
:10A9A00008954EE253E30E9498550895FB01DC019F
:10A9B00004C08D910190801921F441505040C8F796
:10A9C000881B990B0895FB01DC0102C001900D92D8
:10A9D00041505040D8F708956817790768F4FB0193
:10A9E000DC01E40FF51FA40FB51F02C002900E9208
:10A9F00041505040D8F708950C94E354DC0101C055
:10AA00006D9341505040E0F70895FB01DC018D91BA
:10AA100081341CF08B350CF4805E619161341CF044
:10AA20006B350CF4605E861B611189F3990B0895F8
:10AA3000FB01DC010D900020E9F7119701900D92C8
:10AA40000020E1F70895FC018191861721F0882309
:10AA5000D9F7992708953197CF010895FB01DC01BB
:10AA60008D91019080190110D9F3990B0895FB0184
:10AA7000DC0101900D920020E1F70895FB01DC015B
:10AA80004150504088F08D9181341CF08B350CF48E
:10AA9000805E619161341CF06B350CF4605E861B46
:10AAA000611171F3990B0895881BFCCFFB01DC0148
:10AAB0004150504030F08D910190801919F40020E0
:10AAC000B9F7881B990B0895FB01DC0141505040F8
:10AAD00048F001900D920020C9F701C01D9241502D
:10AAE0005040E0F70895FC0181E090E001900616E7
:10AAF00009F4CF010020D1F701970895FB0151918E
:10AB00005523A9F0BF01DC014D9145174111E1F733
:10AB100059F4CD010190002049F04D9140154111AB
:10AB2000C9F3FB014111EFCF81E090E00197089557
:10AB3000FA01A191B081009719F41097E1F0CD01CD
:10AB4000DC01CD010D90002011F4C00113C0FB0108
:10AB50002191222319F02015D9F7F3CFFB01219180
:10AB6000201519F41E92119606C02223C1F70D90EC
:10AB70000020A1F7D001FA01A193B08308950F93AB
:10AB80001F93CF93DF93CDB7DEB72E97CDBFDEBF38
:10AB90000E891F89888D998D26E02C8309831A835D
:10ABA00097FF02C080E090E801978D839E83AE01FD
:10ABB000445E5F4FCE0101966A8D7B8D0E944456A4
:10ABC0004D815E8157FD0AC02F813885421753079A
:10ABD0000CF49A01020F131FF80110822E96CDBFBC
:10ABE000DEBFDF91CF911F910F910895CF93DF9337
:10ABF000CDB7DEB72E97CDBFDEBF85E08C838C89C5
:10AC00009D8989839A83AE01485E5F4FCE0101968C
:10AC10006E897F890E94E3592E96CDBFDEBFDF91FA
:10AC2000CF9108950F931F93CF93DF93CDB7DEB7E6
:10AC30002E97CDBFDEBF8C0186E08C8309831A83FB
:10AC400077FF02C060E070E8615070406D837E83E2
:10AC5000CE010196BA01A9010E9444564D815E8140
:10AC600057FD0AC02F813885421753070CF49A010B
:10AC7000020F131FF80110822E96CDBFDEBFDF91A9
:10AC8000CF911F910F9108952F923F924F925F9213
:10AC90006F927F928F929F92AF92BF92CF92DF92EC
:10ACA000EF92FF920F931F93CF93DF93CDB7DEB751
:10ACB0002D97CDBFDEBF3C016C877D875A01FC011B
:10ACC00016821782838181FFC8C12E010894411C1E
:10ACD000511CF3019381EC85FD8593FD859193FFD4
:10ACE0008191EC87FD87882309F4B3C1853241F453
:10ACF00093FD859193FF8191EC87FD87853229F43F
:10AD000090E0B3010E94745BE4CFFF24EE2410E0D6
:10AD10001032B0F48B3269F08C3228F4803251F06A
:10AD2000833271F40BC08D3239F0803349F41160F5
:10AD30002CC01260146029C0186027C0106125C0A3
:10AD400017FD2EC0282F20532A3098F416FF08C074
:10AD50008F2D880FF82EFF0CFF0CF80EF20E15C089
:10AD60008E2D880FE82EEE0CEE0CE80EE20E10622F
:10AD70000CC08E3221F416FD6CC1106406C08C36F6
:10AD800011F4106802C0883659F4EC85FD8593FDF6
:10AD9000859193FF8191EC87FD87882309F0B8CFD7
:10ADA000982F9554933018F09052933038F424E053
:10ADB00030E0A20EB31E3FE339830FC0833631F07B
:10ADC000833781F0833509F05AC022C0F5018081B4
:10ADD000898322E030E0A20EB31E21E0C22ED12CE6
:10ADE000420114C092E0292E312C2A0C3B1CF501A3
:10ADF0008080918016FF03C06F2D70E002C06FEF5E
:10AE00007FEFC4010E94295B6C0151011F7715C0BF
:10AE100082E0282E312C2A0C3B1CF5018080918089
:10AE200016FF03C06F2D70E002C06FEF7FEFC4010B
:10AE30000E941E5B6C011068510113FD1CC006C00E
:10AE400080E290E0B3010E94745BEA948E2D90E062
:10AE5000C816D906A8F30FC0F40117FD859117FF96
:10AE600081914F0190E0B3010E94745BE110EA947C
:10AE70000894C108D108C114D10471F7E7C0843621
:10AE800011F0893651F5F50117FF07C080819181D6
:10AE9000A281B38124E030E008C080819181AA279B
:10AEA00097FDA095BA2F22E030E0A20EB31E012F2D
:10AEB0000F76B7FF08C0B095A095909581959F4FEC
:10AEC000AF4FBF4F0068BC01CD01A2012AE030E0C6
:10AED0000E94BD5BD82ED4183FC0853721F41F7E59
:10AEE0002AE030E020C0197F8F36A9F0803720F4A7
:10AEF000883509F0AEC00BC0803721F0883709F0E3
:10AF0000A8C001C0106114FF09C0146007C014FF7D
:10AF100008C0166006C028E030E005C020E130E03F
:10AF200002C020E132E0F50117FF07C060817181A6
:10AF30008281938144E050E006C06081718180E0AD
:10AF400090E042E050E0A40EB51EA2010E94BD5B5D
:10AF5000D82ED418012F0F7706FF09C00E7FDF14FB
:10AF600030F404FF06C002FD04C00F7E02C01D2D98
:10AF700001C01F2D802F90E004FF0CC0FE01ED0DDD
:10AF8000F11D2081203311F4097E09C002FF06C0A3
:10AF90001E5F05C086789070009709F01F5F802EB5
:10AFA000992403FD12C000FF0DC0FD2C1E1550F4A6
:10AFB000FE0CF11A1E2D06C080E290E0B3010E9443
:10AFC000745B1F5F1E15C0F304C01E1510F4E11A58
:10AFD00001C0EE2484FE0FC080E390E0B3010E9424
:10AFE000745B82FE1FC081FE03C088E590E010C044
:10AFF00088E790E00DC0C40186789070009791F0CA
:10B0000081FC02C080E201C08BE207FD8DE290E08E
:10B01000B3010E94745B06C080E390E0B3010E941C
:10B02000745BFA94DF14C0F3DA94F201ED0DF11DB4
:10B03000808190E0B3010E94745BDD20A9F706C017
:10B0400080E290E0B3010E94745BEA94EE20C1F7C5
:10B0500040CEF3018681978102C08FEF9FEF2D963E
:10B06000CDBFDEBFDF91CF911F910F91FF90EF9089
:10B07000DF90CF90BF90AF909F908F907F906F9018
:10B080005F904F903F902F90089520FD09C0FC01E4
:10B0900023FD05C022FF02C0738362835183408376
:10B0A0000895CF92DF92EF92FF926B017C0144FDF5
:10B0B00010C046FD10C0D601F701AA0FBB1FEE1F3E
:10B0C000FF1F1094D1F7CA0EDB1EEE1EFF1E81E09B
:10B0D00003C083E001C084E0CC0CDD1CEE1CFF1C2F
:10B0E0008150D1F7C20ED11CE11CF11CB601C70181
:10B0F000FF90EF90DF90CF9008950F931F93CF9321
:10B10000DF938C01C8010E94345BEC0197FD08C0FD
:10B110000E94B7540097B1F7CE01B8010E94A05B1E
:10B12000CE01DF91CF911F910F910895AF92BF9201
:10B13000CF92DF92EF92FF920F931F93CF93DF9303
:10B140008C01D62F5A01C22F0E94345B8B3219F02A
:10B150008D3249F4C068D15009F461C0C8010E9421
:10B16000345B97FD5CC0CD7F2C2F2073D1F48033EE
:10B17000C1F4D15009F43EC0C8010E94345B97FD70
:10B1800039C0C260883711F0883549F4C064D150A5
:10B1900089F1C8010E94345B97FF03C02BC0C6FF32
:10B1A000C061CC24DD247601282F2053283080F084
:10B1B000C4FD09C02A3060F0C6FF05C02F7D322FC4
:10B1C0003151363020F0B8010E94A05B10C02750EA
:10B1D000C701B6014C2F0E9451586B017C01C2601F
:10B1E000D15059F0C8010E94345B97FFDDCFC1FDFB
:10B1F00004C015C0CC24DD247601C7FF08C0F0943C
:10B20000E094D094C094C11CD11CE11CF11CC50178
:10B21000B701A6012C2F0E94455881E001C080E0B3
:10B22000DF91CF911F910F91FF90EF90DF90CF9022
:10B23000BF90AF9008954F925F926F927F928F92DE
:10B240009F92AF92BF92CF92DF92EF92FF920F93B5
:10B250001F93CF93DF93CDB7DEB7A097CDBFDEBFEF
:10B260005C01062F7A016901FE01319680E2DF015F
:10B270001D928A95E9F7D50113961C91139760E00A
:10B2800070E020E040E030E04F0181E0682E712C5A
:10B29000F60113FD559113FF51916F01552309F4E8
:10B2A0007BC05E3519F46115710549F1832F90E07B
:10B2B000861797073CF45D3551F15D3219F444234C
:10B2C00001F103C0442309F4252F852F8695869527
:10B2D0008695F401E80FF11D852F8770230102C0C8
:10B2E000440C551C8A95E2F780818429808352178B
:10B2F00051F0521710F45F5FE8CF5150E6CF31E0C4
:10B3000003C041E001C040E06F5F7F4FC1CF4423E5
:10B3100019F08E8180628E83332351F0FE013196C5
:10B32000CE018196208120952193E817F907D1F766
:10B3300011E001C010E0C5010E94345B9C0197FD43
:10B3400023C0869586958695E1E0F0E0EC0FFD1F21
:10B35000E80FF11D408150E0C9018770907002C074
:10B36000559547958A95E2F740FD05C0C901B5019D
:10B370000E94A05B09C0E114F10419F0D7012D93DC
:10B380007D010150B9F602C0112331F4E114F1043A
:10B3900029F0F701108202C0CC24DD24C601A0965A
:10B3A000CDBFDEBFDF91CF911F910F91FF90EF9046
:10B3B000DF90CF90BF90AF909F908F907F906F90D5
:10B3C0005F904F9008955F926F927F928F929F92BD
:10B3D000AF92BF92CF92DF92EF92FF920F931F93A3
:10B3E000CF93DF930F92CDB7DEB77C015B013A01BB
:10B3F000FC01168217829924EFC0812F90E00E94F1
:10B40000B754009721F0C7010E947D58E5C015325E
:10B4100041F4F50103FD359103FF31915F013532B0
:10B4200061F4C7010E94345B97FDE2C0181709F46C
:10B43000D3C0B7010E94A05BDDC03A3241F403FDE6
:10B44000359103FF31915F015524539401C0552478
:10B45000882410C0F2E05F2A682D70E080E090E060
:10B4600040E20E945158862EF50103FD359103FFFD
:10B4700031915F01232F20532A3060F351FE03C026
:10B48000882019F4B7C088248A94383619F03C36DD
:10B4900099F40AC0F50103FD359103FF31915F0175
:10B4A000383651F4F8E05F2A44E0542AF50103FDF0
:10B4B000359103FF31915F01332309F49BC08BE980
:10B4C0009EE0632F70E039830E94135B39810097FF
:10B4D00009F490C0852D50FC08C0F3010081118152
:10B4E00042E050E0640E751E02C000E010E03E36FF
:10B4F00051F4F7014681578160E070E0C801252DC5
:10B500000E94455869C0333691F481FD02C08824F9
:10B510008394C7010E94345B97FD6AC00115110531
:10B5200019F0F80181938F018A9499F753C0C701EC
:10B530003B3551F4682DA80195010E941B595C010F
:10B54000009709F047C041C039830E947D58398176
:10B5500097FD4EC03F3661F1303728F4343629F17B
:10B56000393649F52AC0333719F0353721F51DC072
:10B57000C7010E94345B6C0197FD11C00E94B75453
:10B58000009729F0C601B7010E94A05B08C0011511
:10B59000110519F0F801C1928F018A9449F701153C
:10B5A0001105C1F0F801108215C0F0E25F2A05C054
:10B5B00040E1542A02C050E4552AC701682DA80171
:10B5C000252D0E949658882329F4F70183818073E2
:10B5D00079F410C050FE9394F7010381F50103FD47
:10B5E000159103FF11915F01112309F006CF02C0ED
:10B5F000992019F0892D90E002C08FEF9FEF0F90F6
:10B60000DF91CF911F910F91FF90EF90DF90CF903E
:10B61000BF90AF909F908F907F906F905F900895B4
:10B62000992788270895FC010590061621F000202F
:10B63000D9F7C00108953197CF010895FC01059015
:10B64000615070400110D8F7809590958E0F9F1F24
:10B650000895FC016150704001900110D8F7809569
:10B6600090958E0F9F1F0895CF93DF93EC012B8150
:10B6700020FF35C026FF09C02F7B2B838E819F8141
:10B6800001968E839F838A8128C022FF0FC0E881A4
:10B69000F9818081992787FD9095009719F42062A0
:10B6A0002B831DC03196E883F98311C0EA85FB85A1
:10B6B000CE01199597FF0BC02B813FEF8F3F93076A
:10B6C00011F480E101C080E2822B8B8308C02E81BF
:10B6D0003F812F5F3F4F2E833F8390E002C08FEF6B
:10B6E0009FEFDF91CF9108950F931F93CF93DF9337
:10B6F0008C01EB018B8181FF1BC082FF0DC02E816D
:10B700003F818C819D812817390764F4E881F98194
:10B710000193E883F98306C0E885F985802F1995A0
:10B72000009731F48E819F8101968E839F8302C0A2
:10B730000FEF1FEFC801DF91CF911F910F91089577
:10B74000FB01238120FF13C026FD11C03FEF8F3F77
:10B75000930781F08283922F90649F7D938326814B
:10B760003781215030402683378390E008958FEF52
:10B770009FEF08958FEF9FEF0895FA01AA272830D1
:10B7800051F1203181F1E8946F936E7F6E5F7F4FAE
:10B790008F4F9F4FAF4FB1E03ED0B4E03CD0670F2A
:10B7A000781F891F9A1FA11D680F791F8A1F911D7D
:10B7B000A11D6A0F711D811D911DA11D20D009F4CD
:10B7C00068943F912AE0269F11243019305D31930F
:10B7D000DEF6CF010895462F4770405D4193B3E0F8
:10B7E0000FD0C9F7F6CF462F4F70405D4A3318F09F
:10B7F000495D31FD4052419302D0A9F7EACFB4E050
:10B80000A6959795879577956795BA95C9F7009707
:10B810006105710508959B01AC010A2E06945795A8
:10B82000479537952795BA95C9F7620F731F841FFF
:0AB83000951FA01D0895F894FFCFA6
:10B83A0000257320257300252D3230732025730DC2
:10B84A000A006F6B006572720025733B25640D0A4E
:10B85A0000257320256420282573290D0A0020203D
:10B86A0020002573202D2068657864756D70286C1A
:10B87A00656E3D2564293A0D0A002530347820206A
:10B88A0000253032782000257325730D0A00082020
:10B89A0008000D0A002000636F6D6D616E64206EF2
:10B8AA006F7420666F756E643A25730D0A002573EE
:10B8BA002000256300240068656C70007072696E50
:10B8CA0074207468697320696E666F726D61746939
:10B8DA006F6E002573202D2068657864756D702859
:10B8EA006C656E3D2564293A0A0D002530347820AE
:10B8FA002000253032782000202020003A20002025
:10B90A00202025730A0D00737563636573730075D0
:10B91A006E6B6E6F776E00616C7265616479206917
:10B92A006E207573650061626F7274656400737965
:10B93A006E63206572726F720063616E63656C6517
:10B94A00642062792072656D6F74650069676E6F35
:10B95A007265640074696D656F75740070726F74D6
:10B96A006F636F6C206572726F72006469736162D3
:10B97A006C65640062757379007265747279206C03
:10B98A0061746572006261642073697A65006F751B
:10B99A0074206F662072616E6765006F70657261F0
:10B9AA0074696F6E206E6F7420737570706F727425
:10B9BA006564006E6F207065726D697373696F6E6E
:10B9CA0000696E636F6D70617469626C6520747969
:10B9DA0070650070617468206E6F7420666F756E92
:10B9EA00640070617273696E67206572726F7200AB
:10B9FA00696E76616C6964207374617465006E6F38
:10BA0A007420636F6E6E6563746564006F7574206D
:10BA1A006F66206D656D6F72792F627566666572E5
:10BA2A007300696E76616C696420706172616D651C
:10BA3A007465727300756E6B6E6F776E20666169DE
:10BA4A006C7572650073772076657273696F6E3AEA
:10BA5A0025642E25642E25640D0A00636F6E6E5FC1
:10BA6A00636220736F636B69643A256420636F6E47
:10BA7A006E65637465643A25640D0A0075736167BF
:10BA8A00653A207365745F706F6C6C5F706572697C
:10BA9A006F64203C706572696F6420696E206D73F3
:10BAAA003E0D0A00706572696F642025640D0A00F4
:10BABA0075736167653A207365745F68656172744E
:10BACA0062656174203C307C313E0D0A00757361F9
:10BADA0067653A207365745F6C6564203C307C311D
:10BAEA003E0D0A00636170733A3078253032780D62
:10BAFA000A00756E6B6E6F776E00667720766572D8
:10BB0A0073696F6E3A25642E25642E25642062754A
:10BB1A00696C643A25730D0A006877207265766944
:10BB2A0073696F6E3A25730D0A0000687474705F4A
:10BB3A00706F7374004C697374656E696E67206FF9
:10BB4A006E2025733A25642F25730D0A00757361DB
:10BB5A0067653A2066775F75706772616465203C35
:10BB6A006D6574686F642C20652E672E20226874B8
:10BB7A0074705F706F7374223E205B3C69703E2064
:10BB8A003C706F72743E203C706174683E5D0D0AB1
:10BB9A00006F6B00657272002573202564202800EF
:10BBAA0069703A257320006D61736B3A2573200022
:10BBBA0067773A25732000646E733A2573290D0A54
:10BBCA0000706565723A25730D0A007573616765C1
:10BBDA003A206765745F7065657261646472203CBF
:10BBEA00736F636B69643E0D0A0073656E64696EF8
:10BBFA006720256420627974657320746F20257329
:10BC0A003A25640D0A0077726F74653A25642072CA
:10BC1A00656D61696E3A25640D0A00757361676521
:10BC2A003A2073656E64746F203C736F636B69644A
:10BC3A003E203C69703E203C706F72743E203C642A
:10BC4A00617461202E2E2E3E0D0A0073656E6469A2
:10BC5A006E672025642062797465730D0A00757316
:10BC6A006167653A2073656E64203C736F636B6924
:10BC7A00643E203C64617461202E2E2E3E0D0A0023
:10BC8A0075736167653A20636C6F7365203C736FE7
:10BC9A00636B69643E0D0A0075736167653A2063D8
:10BCAA006F6E6E656374203C736F636B69643E20CC
:10BCBA003C69703E203C706F72743E0D0A007573C9
:10BCCA006167653A206C697374656E203C736F63B3
:10BCDA006B69643E205B6261636B6C6F675D0D0A22
:10BCEA00006C697374656E5F636220736F636B695E
:10BCFA00643A25642C20616363657074696E6720F9
:10BD0A002E2E2E200028636F6E6E656374696F6E27
:10BD1A00206C6F73742900726563765F63622073A7
:10BD2A006F636B69643A2564206C656E3A256420FA
:10BD3A0025730D0A0052580075736167653A2062CF
:10BD4A00696E64203C736F636B69643E203C697062
:10BD5A003E203C706F72743E0D0A00737472656106
:10BD6A006D00646772616D00726177007573616757
:10BD7A00653A20736F636B6574203C7374726561F6
:10BD8A006D7C646772616D7C7261773E205B707254
:10BD9A006F746F636F6C5D0D0A0075736167653A46
:10BDAA00207365745F6468637064203C307C313E44
:10BDBA000D0A0025732025642028656E61626C6572
:10BDCA00643A2564290D0A0075736167653A207320
:10BDDA0065745F64686370203C307C313E0D0A00F4
:10BDEA0075736167653A207365745F69706164642D
:10BDFA0072203C69703E205B6D61736B5D205B67EE
:10BE0A00775D205B646E735D0D0A004E2F4100253D
:10BE1A0073202564000D0A0020282573202530325E
:10BE2A00783A253032783A253032783A25303278E5
:10BE3A003A253032783A25303278200072737369A5
:10BE4A003A25642000727373693A4E2F41200073B9
:10BE5A006E723A256400736E723A4E2F4100290DB4
:10BE6A000A0025732025642028253032783A2530A7
:10BE7A0032783A253032783A253032783A253032DB
:10BE8A00783A25303278290D0A0075736167653A68
:10BE9A00207365745F6368616E6E656C203C6368CD
:10BEAA00616E6E656C3E0D0A0075736167653A20B6
:10BEBA00636F6E665F6170203C68696464656E3E9C
:10BECA00203C626561636F6E5F696E74766C3E0DCD
:10BEDA000A0020202020202020202020202020208E
:10BEEA00203C696E6163745F746D6F3E205B636FA3
:10BEFA00756E7472795D3E0D0A0075736167653AF5
:10BF0A0020636F6E665F7073203C7573655F707334
:10BF1A005F706F6C6C3E203C70735F747261666612
:10BF2A0069635F74696D656F75743E0D0A00202040
:10BF3A00202020202020202020202020203C707338
:10BF4A005F64656C61793E203C72785F616C6C5FFE
:10BF5A006474696D3E203C6C697374656E5F696ECA
:10BF6A0074657276616C3E0D0A0075736167653A95
:10BF7A00207365745F7073203C307C313E0D0A007B
:10BF8A00257320256420282573290D0A00757361FD
:10BF9A0067653A207365745F777073203C307C3133
:10BFAA003E0D0A0077706132007770610077657024
:10BFBA000075736167653A206C696E6B7570205BFA
:10BFCA00737369645D205B6B65795D205B7765706F
:10BFDA007C7770617C777061325D0D0A00757361E0
:10BFEA0067653A207365745F62617564726174652E
:10BFFA00203C62617564726174653E205B72747381
:10C00A006374735D0D0A00657272202564202866C8
:10C01A0061696C656420746F20636F6E6669677509
:10C02A00726520686F73742075617274290D0A0035
:10C03A004253534944202020202020202020202021
:10C04A002020205459504520202043482052535341
:10C05A004920534E52202041555448202020202068
:10C06A0020535349440D0A002D2D2D2D2D2D2D2DF4
:10C07A002D2D2D2D2D2D2D2D2D2D2D2D2D2D2D2DE6
:10C08A002D2D2D2D2D2D2D2D2D2D2D2D2D2D2D2DD6
:10C09A002D2D2D2D2D2D2D2D2D2D2D2D2D2D2D2DC6
:10C0AA002D2D2D2D2D2D2D2D2D2D2D2D2D0D0A0026
:10C0BA0075736167653A207363616E205B73736998
:10C0CA00645D0D00494E465241004144484F4300C9
:10C0DA00253032783A253032783A253032783A2586
:10C0EA003032783A253032783A25303278202000BA
:10C0FA002573202025303264202530326420200028
:10C10A0025303264202020004E2F412020004E4F3F
:10C11A004E45202020202020005745502020202056
:10C12A00202020005750412D50534B2020200057EB
:10C13A005041322D50534B2020005750412020208F
:10C14A00202020200057504132202020202020008B
:10C15A002573006C6F6F6B75705F63623A20686F4E
:10C16A007374206E6F7420666F756E640D0A006CAE
:10C17A006F6F6B75705F63622069703A25730D0A81
:10C18A000075736167653A206765745F686F7374D9
:10C19A0062796E616D65203C646E736E616D653E99
:10C1AA000D0A00737461006170006164686F630056
:10C1BA0075736167653A207365745F6D6F64652096
:10C1CA003C7374617C61707C6164686F637C7770B6
:10C1DA00733E0D0A007363616E00776C705F736360
:10C1EA00616E287373696429007365745F706F6C7C
:10C1FA006C5F706572696F6400776C705F736574E9
:10C20A005F706F6C6C5F706572696F642829007368
:10C21A0065745F68656172746265617400776C70D9
:10C22A005F7365745F6865617274626561742829F9
:10C23A00007365745F6C656400776C705F73657416
:10C24A005F6C65642829006765745F66775F636160
:10C25A007073007072696E74206669726D776172AC
:10C26A0065206361706162696C69746965730067EE
:10C27A0065745F66775F76657273696F6E00707258
:10C28A00696E74206669726D77617265207665726F
:10C29A0073696F6E006765745F76657273696F6E36
:10C2AA00007072696E7420636C69656E74207665BD
:10C2BA007273696F6E0066775F7570677261646525
:10C2CA0000776C705F66775F757067726164652866
:10C2DA006D6574686F642C20616464722C20706FC1
:10C2EA0072742C207061746829006765745F686FC6
:10C2FA00737462796E616D6500776C705F676574DF
:10C30A005F686F737462796E616D6528646E736EAF
:10C31A00616D6529006765745F7065657261646443
:10C32A007200776C705F6765745F706565726164CF
:10C33A00647228736F636B6964290073656E647431
:10C34A006F00776C705F73656E64746F28736F63C8
:10C35A006B69642C20646174612C2069702C2070D4
:10C36A006F7274290073656E6400776C705F736511
:10C37A006E6428736F636B69642C2064617461292D
:10C38A0000636C6F736500776C705F636C6F7365C5
:10C39A0028736F636B69642900636F6E6E656374DB
:10C3AA0000776C705F636F6E6E65637428736F637A
:10C3BA006B69642C2069702C20706F727429006C70
:10C3CA00697374656E00776C705F6C697374656EFF
:10C3DA0028736F636B69642C206261636B6C6F678F
:10C3EA00290062696E6400776C705F62696E642806
:10C3FA00736F636B2C2069702C20706F7274290024
:10C40A00736F636B657400776C705F736F636B65D2
:10C41A007428747970652C2070726F746F29007398
:10C42A0065745F646863706400776C705F736574C9
:10C43A005F64686370642829006765745F64686371
:10C44A007000776C705F6765745F64686370282931
:10C45A00007365745F6468637000776C705F7365FE
:10C46A00745F6468637028656E61626C6529006731
:10C47A0065745F69706164647200776C705F676588
:10C48A00745F6970616464722829007365745F69F6
:10C49A00706164647200776C705F7365745F697051
:10C4AA00616464722869702C206D61736B2C20673B
:10C4BA00772C20646E7329006765745F6E657477E4
:10C4CA006F726B00776C705F6765745F6E65747707
:10C4DA006F726B2829006765745F6877616464729C
:10C4EA0000776C705F6765745F687761646472284F
:10C4FA0029007365745F6368616E6E656C00776CA2
:10C50A00705F7365745F6368616E6E656C2829007D
:10C51A00636F6E665F617000776C705F636F6E66E3
:10C52A005F6170282900636F6E665F707300776CB5
:10C53A00705F636F6E665F70732829007365745F3E
:10C54A00707300776C705F7365745F70732829006D
:10C55A006765745F6D6F646500776C705F6765749B
:10C56A005F6D6F64652829007365745F6D6F64651C
:10C57A0000776C705F7365745F6D6F64652829005E
:10C58A007365745F77707300776C705F7365745F3F
:10C59A007770732829006765745F6C696E6B6374C2
:10C5AA007800776C705F6765745F6C696E6B5F6348
:10C5BA006F6E746578742829007365745F6C696E90
:10C5CA006B63747800776C705F7365745F6C696E07
:10C5DA006B5F636F6E746578742829006C696E6B83
:10C5EA00646F776E00776C705F6C696E6B646F77DF
:10C5FA006E2829006C696E6B757000776C705F6CC1
:10C60A00696E6B757028737369642C206B65792C5D
:10C61A00206175746829007365745F62617564725C
:10C62A0061746500776C705F7365745F62617564CD
:10C63A00726174652829000D0A0047455420002DAF
:10C64A002D2D2025732070696E67207374617469BB
:10C65A007374696373202D2D2D0A0D0025642070D3
:10C66A0061636B657473207472616E736D6974743F
:10C67A0065642C2025642072656365697665640AA1
:10C68A000D0025642062797465732066726F6D20CF
:10C69A0025733A2069636D705F7365713D25640A7D
:10C6AA000D0025642062797465732066726F6D20AF
:10C6BA0025733A2069636D705F7365713D25642047
:10C6CA0044657374696E6174696F6E20486F737420
:10C6DA0020556E726561636861626C650A0D00259A
:10C6EA00642062797465732066726F6D2025733ACF
:10C6FA002069636D705F7365713D2564205479709C
:10C70A00653A25640A0D006F6B00657272002D632D
:10C71A00002D7300257320256420282573290A0D0E
:10C72A000075736167653A2070696E67205B2D63D7
:10C73A00203C636F756E743E5D205B2D73203C73E5
:10C74A00697A653E5D203C69703E0A0D0070696E2B
:10C75A0067000A0D0074746370206572723A25646A
:10C76A0020282573290A0D0074746370206F6B3AB0
:10C77A0020256C752062797465732070726F636509
:10C78A007373656420696E20256C75206D732C2087
:10C79A00256C75204B422F730A0D00747463702048
:10C7AA006F6B3A20256C75206279746573207072FC
:10C7BA006F63657373656420696E2030206D730A38
:10C7CA000D002E002D70002D6E002D6C002D7400B2
:10C7DA002D7200257320256420282573290A0D004F
:10C7EA00657272007474637020636F6E6E65637431
:10C7FA002025733A2564206E6275663A25642062A4
:10C80A0075666C656E3A256420736F636B69643A6A
:10C81A0025640A0D0074746370206C697374656E04
:10C82A0020706F72743A2564206275666C656E3A80
:10C83A002564206C736F636B69643A25640A0D0082
:10C84A0075736167653A2074746370205B2D747226
:10C85A00706E6C5D0A0D007474637000747463709A
:10C86A00207468726F756768707574207465737464
:10C87A00006661696C656420746F20676574206E58
:10C88A0074702074696D653A2573282564290A0D28
:10C89A00006E74702074696D653A20253034642DF9
:10C8AA00253032642D2530326420253032643A2511
:10C8BA003032643A253032640A0D006F6B006572BB
:10C8CA007200257320256420282573290A0D007516
:10C8DA00736167653A206E7470203C6E74702D73B4
:10C8EA0065727665723E0A0D0000001F003B005A11
:10C8FA000078009700B500D400F300110130014E12
:10C90A00016D0100001F003C005B0079009800B631
:10C91A0000D500F400120131014F016E016E7470EE
:10C92A0000676574207365727665722074696D6537
:10C93A002066726F6D206E7470004E2F4100253094
:10C94A0032783A253032783A253032783A25303200
:10C95A00783A253032783A25303278002F002F3F46
:10C96A00002F696E6465782E68746D6C3F00746F71
:10C97A0067676C653D4C45442564002F696E6465A4
:10C98A00782E68746D6C002F6C6F676F2E676966FE
:10C99A00006C696E6B5F6362206C696E6B3A25642A
:10C9AA000A0D006669726D7761726520757067722B
:10C9BA0061646520636F6D706C6574650A0D00664D
:10C9CA0069726D776172652075706772616465203E
:10C9DA006661696C65640A0D00616464725F636212
:10C9EA002069703A6E6F6E650A0D00616464725F49
:10C9FA0063622069703A25730A0D00686477697268
:10CA0A00656C657373006864776972656C657373C6
:10CA1A0031323300004E0045004F004D00530000F4
:10CA2A000027342000FFFFFFFF000000008720C01E
:10CA3A00188C20E720F620FE2009211C2124212C15
:10CA4A00213B214421492155215E216B21832191DA
:10CA5A0021A321B221C021CE21DC21F2210522A568
:10CA6A0029E530AA29B9293723C929DF29CB23ED9A
:10CA7A0029012A2D24092A172A6324232A3F2A92C4
:10CA8A00244E2A652AA922712A862A1125912ABAB0
:10CA9A002AC432C92AE52A8326F22A0B2BDF261258
:10CAAA002B352BCD273A2B512B8B28572B692BC192
:10CABA0028712B8F2B1729962BB22B152AB72BD01F
:10CACA002B6B2AD72BEF2BE82AF92B092C1E2B12BA
:10CADA002C212C5C2B2A2C3F2CCA254A2C5B2C920D
:10CAEA002B662C882C1C2C942CA62C3D2DB12CC2E8
:10CAFA002C8A2DCE2CE02CC32DE82CF62C302EFEC1
:10CB0A002C0C2DBD2E132D202DF32E292D382DEA78
:10CB1A0032412D502D3D2F582D662D732F722D89A0
:10CB2A002D842F952DAC2D922FB52DC42D9E2FCB54
:10CB3A002DE72D3A30F42D732977297A291D2F8470
:10CB4A00361D2F2730563A2C30ED30F43CF13001A7
:0ECB5A00020307E531E731E931EB31ED31003F
:00000001FF
